:100000000C9497030C94B4030C94B4030C94B403B1
:100010000C94B4030C94B4030C94B4030C94B40384
:100020000C94B4030C9480170C94B4030C94B40394
:100030000C94CB2B0C94B4030C94B4030C94B40325
:100040000C94B4030C94B4030C941A160C94B403DB
:100050000C94D6090C94B4030C949F090C94B4032B
:100060000C94571B0C94B4030C94562A0C94B403B0
:100070000C94755D0C94B4030C94B403D71EE31E6A
:10008000801D8C1DA61DA11B4F1D611D9C1CCB1B23
:10009000A11BC01DD11DEB1D0B1E2B1E811EBC1BE9
:1000A000A52A262B122B632B572B412B6C2A6C2A4B
:1000B000862A382BF32A8F2A982A862AE02AD62ADB
:1000C0008F2A982A862A092BE92A8F2AFD2A0A0DC7
:1000D0003D3D3D3D3D3D3D3D3D3D3D3D3D3D3D3D50
:1000E0003D3D3D3D3D3D3D3D3D3D3D3D3D3D3D3D40
:1000F0003D3D3D0A0D004E6F726D616C20284143FD
:10010000432D4D6F6465290048656164696E6748D9
:100110006F6C64000A0D436F6E74726F6C3A20004E
:100120004F4B0A0D000A0D43616C6962726174697C
:100130006E672070726573737572652073656E7378
:100140006F722E2E000A0D5573696E6720706172F2
:10015000616D65746572736574202564000A0D41D4
:100160004343206E6F742063616C696272617465D1
:10017000642021003A2047656E65726174696E677C
:100180002044656661756C742D506172616D657493
:100190006572207573696E67206F6C642053746993
:1001A000636B2053657474696E6773000A0D496E42
:1001B00069742E20454550524F4D000A0D3D3D3D7E
:1001C0003D3D3D3D3D3D3D3D3D3D3D3D3D3D3D3D5F
:1001D0003D3D3D3D3D3D3D3D3D3D3D3D3D3D3D3D4F
:1001E000000A0D0A0D2121204D495353494E472045
:1001F000424C2D4354524C3A2025642021210025A5
:100200006420000A0D466F756E6420424C2D4374C5
:10021000726C3A20000A0D4D697865722D436F6E3D
:100220006669673A202725732720282575204D6F9A
:10023000746F727329000A0D47656E657261746987
:100240006E672064656661756C74204D69786572AF
:10025000205461626C65000A0D466C6967687443DE
:100260006F6E74726F6C0A0D4861726477617265AB
:100270003A25642E25640A0D536F667477617265A2
:100280003A5625642E2564256320000A0D3D3D3D28
:100290003D3D3D3D3D3D3D3D3D3D3D3D3D3D3D3D8E
:1002A0003D3D3D3D3D3D3D3D3D3D3D3D3D3D3D3D7E
:1002B000000A0D20444143206F72204932432045FB
:1002C00052524F522120436865636B204932432CC0
:1002D0002033567265662C2044414320616E6420B1
:1002E000424C2D4374726C002E00313200313100CB
:1002F0003130002025632020202D2020202D20209B
:10030000202D002025632020202563202020256328
:100310002020202563200020256320202025632025
:100320002020256320202025632000424C2D43748B
:10033000726C20666F756E64200020253364202067
:1003400025336420202533642020253364200020B9
:100350002533642020253364202025336420202584
:100360003364200020253364202025336420202599
:10037000336420202533642000424C2D4374726C7A
:10038000204572726F7273200048693A25346920E3
:100390002043663A253469200047733A25346920A2
:1003A0002047693A25346920004E693A253469208E
:1003B00020526F3A253469200045787465726E4387
:1003C0006F6E74726F6C20200052616E67653A2503
:1003D00033692D253369005374656C6C756E673A0B
:1003E0002025336900536574706F696E7420202571
:1003F000336900536572766F202000506F74693442
:100400003A202025336900506F7469333A20202543
:10041000336900506F7469323A20202533690050E7
:100420006F7469313A202025336900537461727406
:100430003A2020202020253569004D6573737765AB
:1004400072743A2020253569005269636874756EAC
:10045000673A2020253569004B6F6D7061737320FA
:1004600020202020202000456D70662E5065676595
:100470006C3A253569005370616E6E756E673A206F
:100480002025356900486F636820253469202825B8
:1004900033692900526F6C6C20253469202825337C
:1004A0006929004E69636B2025346920282533694A
:1004B0002900414343202D2053656E736F7200471E
:1004C0006965722025346920282533692928253358
:1004D000692900526F6C6C20253469202825336906
:1004E000292825336929004E69636B20253469204A
:1004F0002825336929282533692900476965722031
:1005000025346920282533692900526F6C6C202519
:10051000346920282533692E257829004E69636BBC
:100520002025346920282533692E2578290047693C
:1005300065722025346920282533692900526F6CA3
:100540006C2025346920282533692E256929004E21
:1005500069636B2025346920282533692E25692994
:10056000004779726F202D2053656E736F720050B3
:10057000333A253469202050343A2534692000501C
:10058000313A253469202050323A25346920004719
:10059000733A253469202047693A25346920004E92
:1005A000693A2534692020526F3A25346920004B7E
:1005B000373A25346920204B383A25346920004BDE
:1005C000353A25346920204B363A25346920004BD2
:1005D000333A25346920204B343A25346920004BC6
:1005E000313A25346920204B323A25346920004BBA
:1005F0006F6D706173733A20202025356900526F4A
:100600006C6C3A202020202020253569004E69633B
:100610006B3A20202020202025356900616B742E44
:10062000204C6167650048F668656E726567656CA9
:10063000756E67004B65696E6520004F6666202009
:10064000202020203A20253569004C75667464729C
:1006500075636B3A2025356900536F6C6C486F6584
:1006600068653A2025356900486F6568653A20203D
:100670002020202535690028632920486F6C676594
:10068000722042757373004D697373696E672042FF
:100690004C2D4374726C3A25642121004932432069
:1006A0004552524F522121210053657474696E677F
:1006B0003A25642025730048573A5625642E256450
:1006C0002053573A25642E25642563002B204D695D
:1006D0006B726F4B6F70746572202B005B25695DC8
:1006E000005B25695D0054696D656F75742E0A0D98
:1006F000006F6B2E0A0D000A0D506C65617365204A
:10070000636F6E6E656374205370656B7472756D84
:1007100020726563656976657220666F7220626912
:100720006E64696E67204E4F572E2E2E00001124E6
:100730001FBECFEFD0E1DEBFCDBF13E0A0E0B1E040
:10074000EAE2F4EC02C005900D92AE3CB107D9F795
:1007500019E0AEECB3E001C01D92AF38B107E1F78C
:100760000E94AB040C9413620C9400009C01F99954
:10077000FECF32BD21BDF89A80B508959C01F9994C
:10078000FECF1FBA32BD21BD60BD0FB6F894FA9AF4
:10079000F99A0FBE0895F999FECF22E030E032BDFC
:1007A00021BDF89A90B5892F8150853068F0F9996C
:1007B000FECF1FBA32BD21BD83E080BD0FB6F894D5
:1007C000FA9AF99A0FBE93E0892F0895282F863060
:1007D00078F025E0F999FECF1FBA82E090E092BD53
:1007E00081BD20BD0FB6F894FA9AF99A0FBE08950C
:1007F000882381F7089580916008A82FB0E0AA0FA0
:10080000BB1FFD01E25DF74F808191818D5E9F4F9F
:1008100014F010920A01A25DB74F8D919C918A5BF2
:100820009F4FA4F480910A01882381F481E0809392
:100830000A018091FB068F5F8093FB06853068F08C
:1008400088EE93E09093EF038093EE038091FB0694
:100850008093C8071092C90708950E94453E809171
:10086000FB068093C8071092C90708950F931F9342
:10087000CF93DF93082FEB01142F863008F43FC08D
:1008800005E024E030E0812F90E0AC01249FC0011E
:10089000259F900D349F900D11248C599F4FBE01C0
:1008A000412F50E02EEB33E00E94E15FF999FECF3B
:1008B0001FBA82E690E092BD81BD10BD0FB6F894DC
:1008C000FA9AF99A0FBE4297BE0148E050E02EEB2B
:1008D00033E00E94E15FF999FECF1FBA82E090E019
:1008E00092BD81BD00BD0FB6F894FA9AF99A0FBE79
:1008F0000E94995CDF91CF911F910F9108958823F9
:1009000029F4DF91CF911F910F910895282F30E0A6
:1009100021503040B8CF982FFB0181508530B0F086
:1009200022E030E0842F90E0289FB001299F700DD5
:10093000389F700D11246C597F4FCF0150E026EB8A
:1009400033E00E94C55F0E94995C0895292F30E032
:1009500021503040E7CF2F923F924F925F926F929B
:100960007F928F929F92AF92BF92CF92DF92EF923F
:10097000FF920F931F93CF93DF9314B815B8189B72
:10098000A9C3199BC7C48DE08093080181E887B98A
:100990003E9A8FEF88B98BE184B981E085B98EE307
:1009A0008AB9579A87E48BB9469A84B7877F84BF00
:1009B000809160008861809360001092600080EDFB
:1009C00097E09093EF038093EE031092A5041092AA
:1009D000A40410923308109232081092A3041092CB
:1009E000A2041092A1041092A004209108012431C5
:1009F00008F463C388E894E0A0E0B0E08093BD030E
:100A00009093BE03A093BF03B093C0032A3009F4B0
:100A100052C3243109F44FC3289A0E9468170E94D8
:100A200040170E94780B0E94B62B0E94511B0E9417
:100A30000C2A0E945559789400D00F92ADB7BEB7DA
:100A400011961C9211978BE892E013969C938E93CB
:100A500012970E94E21220910801EDB7FEB73A9773
:100A60000FB6F894FEBF0FBEEDBF3196ADB7BEB75F
:100A700011961C9287E592E092838183822F6AE02F
:100A80000E946C6183831482822F0E946C61958323
:100A90001682108617828AE490E0928781878FEC15
:100AA0009DE4948783870E94E2128091C800EDB78D
:100AB000FEB73D960FB6F894FEBF0FBEEDBF803275
:100AC00009F420C4809108018C3008F0F2C2299A00
:100AD00083E060E678E049E00E948B04F999FECF5C
:100AE00088EE93E092BD81BDF89A80B5813009F41B
:100AF0005BC000D00F92ADB7BEB711961C92119794
:100B000086E392E013969C938E9312970E94E212D2
:100B1000EDE5F5E00F900F900F9010821182128298
:100B200013823496B5E0ED39FB07B9F780E4809382
:100B30005D05FF97808310925F0580936005809329
:100B4000610590EC909362051092630580936405B3
:100B500080936505109266059093670590936805EC
:100B60008093690510926A0580936B0590936C05DC
:100B700081E080935005EF012D97DE01E0E0F1E088
:100B80008BE001900D928150E1F788EE93E060E5F3
:100B900075E04DE450E02EEB33E00E94E15F11E0A0
:100BA000E12E10E0F12E2AC0F999FECF01E0E02EEF
:100BB00000E0F02EF2BCE1BCF89A80B58F3F09F45A
:100BC00098CF1092C10380E595E068EE73E04DE4A4
:100BD00050E026EB33E00E94C55FEDE5F5E0808153
:100BE00018162CF48091C1038F5F8093C103349653
:100BF00025E0ED39F20799F7C1E5D5E0EDB7FEB78D
:100C000037970FB6F894FEBF0FBEEDBF3196ADB764
:100C1000BEB711961C9285E192E092838183D483C2
:100C2000C3838091C103858316820E94E2120F90D4
:100C30000F900F900F90EDB7FEB7118283E092E016
:100C4000938382830E94E212109233041092EB038A
:100C50000F900F900F900E94F5398091EB0388233D
:100C6000E1F310923304C1E0D0E00FEF11E01092F5
:100C7000EB030E94F5398091EB038823E1F3FE0139
:100C8000EF5DF74F80818823A9F000D000D00F924C
:100C9000EDB7FEB73196ADB7BEB711961C92128371
:100CA0000183D483C3830E94E2120F900F900F90B0
:100CB0000F900F902196CD30D105C9F60DE515E0C6
:100CC000C1E0D0E0B1EECB2EB1E0DB2EFE01EF5D56
:100CD000F74F80818823C9F4F80180811816ACF49D
:100CE00000D000D00F92EDB7FEB73196ADB7BEB7CA
:100CF00011961C92D282C182D483C3830E94E212D5
:100D00000F900F900F900F900F90FE01EB5FF74F39
:100D1000108221960C5F1F4FCD30D105B9F600D05F
:100D20000F92EDB7FEB711828BEB91E09383828334
:100D30000E94E2120F900F900F90F999FECFF2BC33
:100D4000E1BCF89A80B58B3409F484C00E947C58C9
:100D500000D00F92ADB7BEB711961C9211978CEAD6
:100D600091E013969C938E9312970E94E212C0E535
:100D7000D0E011E00F900F900F905E010894A11C3D
:100D8000B11CA2E08A2E912C8C0E9D1EF3E06F2EDA
:100D9000712C6C0E7D1EE4E04E2E512C4C0E5D1E0F
:100DA00075E0272E312C2C0E3D1E64E7C62E61E027
:100DB000D62E05E0123009F409C2133009F463C2DB
:100DC000143008F003C280910801843160F0009370
:100DD000780810929008BBE1B0937408EEE4E093B9
:100DE0008D08E0938E08F999FECFD2BDC1BDF89A67
:100DF00080B58C3048F4F999FECFB2BCA1BCF89A0A
:100E000080B58C3008F46CC10E94B22C812F60E652
:100E100078E04DE50E9436041F5F163008F4CACF13
:100E2000F999FECF1FBA82E090E092BD81BD83E0C8
:100E300080BD0FB6F894FA9AF99A0FBEF999FECFD1
:100E40001FBAF2BCE1BC8BE480BD0FB6F894FA9AED
:100E5000F99A0FBEF999FECF84E090E092BD81BD72
:100E6000F89A80B5853008F03EC20E94CB0360E658
:100E700078E04DE50E948B040E94CB0300D000D0A7
:100E80000F92EDB7FEB73196ADB7BEB711961C9273
:100E900025E431E032832183838314820E94E212AD
:100EA000809168080F900F900F900F900F9080FD29
:100EB000EDC1C8EED3E00E94BD3B809108018A30AD
:100EC00009F4D0C1843109F4CDC1289A80ED97E0AE
:100ED0009093EF038093EE0385E58093FD0600D0A9
:100EE0000F92EDB7FEB7118284E191E09383828384
:100EF0000E94E212809168080F900F900F9082FF7D
:100F0000B3C100D00F92ADB7BEB711961C92119726
:100F100088E091E013969C938E9312970E94E212C0
:100F20000F900F900F9000D00F92ADB7BEB71196F3
:100F30001C9211978EEC90E013969C938E931297CF
:100F40000E94E2120F900F900F900E94DA2088E822
:100F500093E190939E0380939D0381E08093FC0630
:100F600014E050E7852E57E1952E612C43E0742E56
:100F700030E1C32E37E2D32E20E8A22EB12C95E02B
:100F8000E92EF12C8091EB03882309F486C080912F
:100F90002703882309F481C01092EB038091FB069C
:100FA000882309F447C10E94FB030E94F539209170
:100FB00008012A3009F429C1243109F426C1289AEC
:100FC00080910D01882309F426C1815080930D0181
:100FD00080919F04882329F080919F048150809301
:100FE0009F0480913B05882369F0815080933B05E5
:100FF000882341F4109224051092230510922605AF
:101000001092250580919D0390919E0301979093E6
:101010009E0380939D0380919D0390919E03892B55
:1010200009F4D7C080913404882309F0D2C02A3053
:1010300009F40DC1243109F40AC1289A8091EB0307
:10104000882329F08091A804882309F0FDC00E941C
:10105000B80C0E94B50FCE010E94FF168823D9F06C
:1010600020911803309119038091790890E0281796
:10107000390744F480911103909112038F5F9F4FC1
:1010800009F4E7C00E94D05B1093F00384E190E084
:101090000E94F516EC010E94A85C8091F003882361
:1010A00009F070CF0E94115C8091EB038823A9F3B3
:1010B0006ECF29980DCD2898B0CC8BE095E0A0E0BC
:1010C000B0E08093BD039093BE03A093BF03B093A1
:1010D000C0039CCC199B22C184E18093080156CCAB
:1010E000F999FECF92BC81BCF89A80B58C3008F09B
:1010F0008BCEF999FECF72BC61BCF89A80B58C306A
:1011000008F082CEF999FECFD2BDC1BDF89A80B564
:1011100080936008F999FECF21E530E032BD21BD12
:10112000F89A80B580936108F999FECF82E590E046
:1011300092BD81BDF89A80B580936208F999FECF7F
:10114000A3E5B0E0B2BDA1BDF89A80B58093630875
:10115000F999FECF52BC41BCF89A80B580936408DF
:10116000F999FECF32BC21BCF89A80B5809365080E
:10117000F999FECFE6E5F0E0F2BDE1BDF89A80B561
:1011800080936608F999FECF27E530E032BD21BD96
:10119000F89A80B580936708113009F037CE00D0F7
:1011A0000F92ADB7BEB711961C9211971396DC92B1
:1011B000CE9212970E94E2120F900F900F9081E052
:1011C00060E678E04DE50E94360412E00E94CB57BD
:1011D000FACD80919D0390919E03892B71F18091AE
:1011E0001103909112038F5F9F4F09F027CF8091D9
:1011F000A804882309F422CFD092EF03C092EE0313
:10120000B0921203A092110319CF289880910D017A
:10121000882309F0DACE109207071092C0041092CA
:10122000BF041092C2041092C1041092C404109220
:10123000C304CECE0E94673EB8CE0E941A2AF09216
:101240009E03E0929D03CBCF0E94B50F04CF289858
:10125000F5CE9092EF038092EE03709212036092AB
:10126000110310CF289832CE00D00F92EDB7FEB701
:10127000118286EF90E0938382830E94E2120F90A6
:101280000F900F9050CE0E941C579DCD00D00F9212
:10129000EDB7FEB7118285E291E0938382830E94CD
:1012A000E2120F900F900F9088EE93E00E94F516D7
:1012B000EC010E947520CE010E94FF168823D9F30D
:1012C00000D00F92ADB7BEB711961C92119780E275
:1012D00091E013969C938E9312970E94E2120F90C6
:1012E0000F900F90E8CD00D00F92EDB7FEB71182AE
:1012F0008DE591E0938382830E94E2120F900F901C
:101300000F90B3CD8091CA00863009F0DBCB0E94EC
:101310001F5DD8CB8BE08093080138CB8AE08093A7
:10132000080134CB9C01F999FECF1FBA32BD21BD13
:1013300060BD0FB6F894FA9AF99A0FBE08951F92FD
:101340000F920FB60F9211248F939F93EF93FF93F9
:1013500080910B018823A9F48091E7039091E80321
:1013600001969093E8038093E703FC01E355FA4F5D
:10137000E081ED3099F08639910581F0E093C60067
:1013800004C01092E8031092E703FF91EF919F9140
:101390008F910F900FBE0F901F9018951092E80339
:1013A0001092E70381E080930B01E8CF1F920F9228
:1013B0000FB60F9211242F933F934F938F939F93C8
:1013C000AF93BF93CF93DF93EF93FF938091C600CA
:1013D0008093D5034091E203463910F01092E10367
:1013E0008091D5038D3079F18091E103813009F44A
:1013F0009EC08130A8F0823009F481C01092E103D0
:10140000FF91EF91DF91CF91BF91AF919F918F911C
:101410004F913F912F910F900FBE0F901F901895F5
:101420008091D503833209F4A0C08091D5038093C5
:101430000A0781E08093E2038091D5038093E5035E
:101440001092E603DDCF8091E103823079F61092AD
:10145000E103A42FB0E0FD01E85FF84F3081ED011A
:10146000C75FD84F28818091E5039091E603831BE5
:101470009109821B91099F709093E6038093E50385
:101480009C010024220F331F001C220F331F001C5D
:10149000232F302D235C2093E403982F9F73935CBC
:1014A0009093E3038081281709F468C08091D803E2
:1014B0008F5F8093D80390E08091D603882309F052
:1014C0009FCF992309F49CCF81E08093D6034F5F8F
:1014D0004093D903A65FB84F8DE08C9380910C07A1
:1014E000823509F08DCF2CE088E190E00FB6F894BA
:1014F000A895809360000FBE2093600081CFE42FF9
:10150000F0E08091D503E65FF84F8083463948F1DB
:101510001092E1032091D5038091E5039091E603B9
:10152000820F911D9093E6038093E50369CF82E0DB
:101530008093E103E42FF0E08091D503E65FF84F5C
:1015400080834F5F4093E2032091D5038091E503B0
:101550009091E603820F911D9093E6038093E5033B
:101560004FCF4F5F4093E203D5CF8091D6038823BE
:1015700009F05BCF81E08093E10357CF8881981712
:1015800009F094CF91E098CFCF93DF93BC010097FF
:10159000A9F120E030E040E050E0FA01E355FA4FD5
:1015A0008081280F311D4F5F5F4F46175707A8F303
:1015B0003F70C9010024880F991F001C880F991FD4
:1015C000001C892F902D835CDB0111962F73235C07
:1015D000ED012196FB01E355FA4F8083A355BA4FE5
:1015E0002C93C355DA4F8DE0888310920B018091C4
:1015F000AD058093C600DF91CF910895E0E0F0E063
:101600008DE3A1E0B0E02DE3C2E0D0E0E4CF509163
:10161000D903565009F457C033E043E01EC0972F5A
:101620009D53F0E02295207F892F86958695282B63
:10163000E65FF84F2083E42FEE5F5230C1F1535044
:10164000F0E09295990F990F907C6D53962BE65F81
:10165000F84F90834D5F5523A1F1E32FF0E0E65F53
:10166000F84F80813F5FE32FF0E0E65FF84F208185
:101670002D533F5FE32FF0E0E65FF84F70813F5F4F
:10168000E32FF0E0E65FF84F60813F5F922F929585
:101690009F708D53880F880F892BE42FF0E0E65F51
:1016A000F84F8083E42FEF5F513009F0B8CFE3505B
:1016B0008DE097E09093DB038093DA03E093DC0303
:1016C0000895E42FF4CFE0E0F3CF1F93182F8A3072
:1016D00051F08091C00085FFFCCF1093C60080E0E0
:1016E00090E01F9108958DE00E94650BF2CF089560
:1016F000E1ECF0E088E18083A0ECB0E08C918260C6
:101700008C938081806880838081806480838AE27A
:101710008093C40080910F01909110010E94F516F2
:101720009093DA068093D9068CED90E00E94F5162E
:1017300090930907809308071092DB068AE4809350
:10174000DC0683E08093DF068AE08093DD0681E09B
:101750008093DE061092DB031092DA031092DC0312
:101760000895BF92CF92DF92EF92FF920F931F9353
:10177000DF93CF93CDB7DEB78D852E8593E290931F
:10178000AD058F598093AE058C858093AF052223DC
:1017900079F463E070E0CB010E94C40ACF91DF913D
:1017A0001F910F91FF90EF90DF90CF90BF90089521
:1017B000EF84F88803E1C02ED12CCC0EDD1E4989C0
:1017C0005A894115510529F3022F015063E070E059
:1017D00010E062C0A12FB0E01F5FFA01AE0DBF1D87
:1017E0008C91AF014150504009F48BC0E12FF0E0E3
:1017F0001F5FEE0DFF1DA0814150504009F06DC0EC
:10180000002309F46AC096012E5F3F4FF601E08085
:10181000F180B2E0CB2ED12CC20ED31EF901408153
:1018200051810150382F32953F7090E08F70907049
:101830002A2F2295269526952370880F991F880FA9
:10184000991F282B235CAF73A35C10E08B2D86952A
:101850008695835CFB01E355FA4F80838B2D90E0E6
:101860008370907082959295907F9827807F9827BB
:10187000382B335CFB01E255FA4F3083FB01E15515
:10188000FA4F2083FB01E055FA4FA0836C5F7F4F36
:101890004115510509F47FCFF701E10FF11DB0802B
:1018A0001F5F4150504009F095CF002391F0F601A1
:1018B0003296D601ED90FC9012E0C12ED12CCE0EC6
:1018C000DF1E0190F081E02D0150309709F04CC0EF
:1018D00010E030E02DE3ADE3B9CF382F32953F7003
:1018E00090E08F7090702A2F229526952695237070
:1018F000880F991F880F991F282B235CAF73A35C57
:10190000A5CF002371F4382F32953F7090E08F708F
:101910009070880F991F880F991F282F235CADE3C3
:1019200095CFF6013296D601ED90FC90A2E0CA2E3A
:10193000D12CCE0EDF1E4081518101504115510541
:1019400021F0E0E0F0E011E054CF382F32953F7005
:1019500090E08F709070880F991F880F991F282F23
:10196000235C10E0ADE372CFA0E0B0E011E036CF31
:10197000EF92FF920F931F9380910B01882309F43C
:1019800097C08091D003882329F080910B01882390
:1019900009F0CAC08091CF03882329F080910B0100
:1019A000882309F005C18091D203882329F0809112
:1019B0000B01882309F036C18091CE03882329F0DA
:1019C00080910B01882309F056C1809108079091FE
:1019D00009070E94FF16882329F080910B018823B4
:1019E00009F074C180910F0190911001892B09F0C9
:1019F00064C08091D103882329F080910B01882352
:101A000009F07DC28091DF039091E003892B09F0FA
:101A1000F0C120910C012F3FD1F18DB79EB70B97EC
:101A20000FB6F8949EBF0FBE8DBFEDB7FEB73196CF
:101A300081E4ADB7BEB711968C9381E0818382E0DB
:101A400082838CE091E09483838381E090E09683AD
:101A50008583822F90E082959295907F9827807F52
:101A600098278F5E9E4F9087878380E190E09287D2
:101A700081870E94B10B8FEF80930C012DB73EB789
:101A8000255F3F4F0FB6F8943EBF0FBE2DBF80912C
:101A9000E207882329F080910B01882309F080C197
:101AA0008091D303882321F080910B01882379F45E
:101AB0001F910F91FF90EF9008958091D90690911A
:101AC000DA060E94FF16882309F097CF92CF8DB7D0
:101AD0009EB707970FB6F8949EBF0FBE8DBFEDB7A8
:101AE000FEB7319680E5ADB7BEB711968C9381E015
:101AF000818382838EE298E09483838386E190E001
:101B0000968385830E94B10B1092D3032DB73EB705
:101B1000295F3F4F0FB6F8943EBF0FBE2DBF1F91F8
:101B20000F91FF90EF9008950E94E3202DB73EB7EC
:101B30002B5030400FB6F8943EBF0FBE2DBFEDB70F
:101B4000FEB7319688E4ADB7BEB711968C9381E0AD
:101B5000818382E0828384ED93E09483838381E0B8
:101B600090E0968385838091D40324E1829FC00115
:101B700011248E5C9C4F9087878384E190E092874C
:101B800081870E94B10B8091D4038F5F8093D4032F
:101B90002DB73EB7255F3F4F0FB6F8943EBF0FBE3F
:101BA0002DBF843010F01092D4031092D003F2CEE7
:101BB0000E94E3208DB79EB70F970FB6F8949EBF93
:101BC0000FBE8DBFEDB7FEB731968CE4ADB7BEB793
:101BD00011968C9381E0818383E082838FE294E08D
:101BE0009483838321E030E03683258382E893E089
:101BF000908787833287218782E393E09487838766
:101C000080E590E0968785870E94B10B1092CF0304
:101C10002DB73EB7215F3F4F0FB6F8943EBF0FBEC2
:101C20002DBFC1CE8DB79EB707970FB6F8949EBF54
:101C30000FBE8DBFEDB7FEB7319686E5ADB7BEB727
:101C400011968C9381E0818382838BED96E094835F
:101C500083838AE090E0968385830E94B10B109283
:101C6000D2032DB73EB7295F3F4F0FB6F8943EBF62
:101C70000FBE2DBFA1CE8DB79EB707970FB6F894B4
:101C80009EBF0FBE8DBFEDB7FEB7319687E4ADB7EF
:101C9000BEB711968C9380910E01818381E082837F
:101CA0008DEF96E0948383838BE090E09683858329
:101CB0000E94B10B1092CE032DB73EB7295F3F4F64
:101CC0000FB6F8943EBF0FBE2DBF7FCEE0907408D4
:101CD000FF24EE0CFF1CEE0CFF1C0027F7FC009508
:101CE000102F609150047091510480915204909192
:101CF0005304A80197010E94C1613093F606209316
:101D0000F506609158047091590480915A0490919D
:101D10005B04A80197010E94C1613093F8062093EB
:101D2000F7068091B7048093F9068091B8048093F8
:101D3000FA068DB79EB707970FB6F8949EBF0FBEF1
:101D40008DBFEDB7FEB7319687E7ADB7BEB7119639
:101D50008C9383E0818381E0828385EF96E0948396
:101D6000838388E090E0968385830E94B10B2DB732
:101D70003EB7295F3F4F0FB6F8943EBF0FBE2DBF51
:101D80008091FB06853018F086E08093FB0683E6A1
:101D900090E00E94F516909309078093080722CEE1
:101DA0008DB79EB707970FB6F8949EBF0FBE8DBF35
:101DB000EDB7FEB7319682E4ADB7BEB711968C93FE
:101DC00081E08183828382EE97E09483838381E044
:101DD00090E0968385830E94B10B1092E2072DB7A5
:101DE0003EB7295F3F4F0FB6F8943EBF0FBE2DBFE1
:101DF00057CE8091AB059091AC050E94FF168823C9
:101E000009F407CE80910B01882309F402CEE090FB
:101E10007408FF24EE0CFF1CEE0CFF1C0027F7FCDF
:101E20000095102F609150047091510480915204DC
:101E300090915304A80197010E94C16130939E05BF
:101E400020939D05609158047091590480915A0423
:101E500090915B04A80197010E94C1613093A00595
:101E600020939F0560912209709123098091240994
:101E7000909125092AE030E040E050E00E944D6159
:101E80002091BD033091BE034091BF035091C00328
:101E90000E94C1613093A2052093A1058DB79EB722
:101EA00007970FB6F8949EBF0FBE8DBFEDB7FEB774
:101EB000319683E4ADB7BEB711968C9381E08183F0
:101EC00082838DE995E0948383838EE090E096830E
:101ED00085830E94B10B2DB73EB7295F3F4F0FB6E8
:101EE000F8943EBF0FBE2DBF8091DF039091E003B9
:101EF0000E94F5169093AC058093AB058ACD8DB703
:101F00009EB707970FB6F8949EBF0FBE8DBFEDB773
:101F1000FEB7319684E4ADB7BEB711968C9381E0DD
:101F20008183828380EA97E09483838382E490E0D4
:101F3000968385830E94B10B1092D10380910F018B
:101F4000909110012DB73EB7295F3F4F0FB6F8941F
:101F50003EBF0FBE2DBF009709F454CD0E94F51669
:101F60009093DA068093D9064DCDEF92FF920F93AE
:101F70001F93DF93CF9300D0CDB7DEB78091D60308
:101F8000882349F40F900F90CF91DF911F910F910B
:101F9000FF90EF9008950E94070B80910B07823607
:101FA000F1F180910C07843609F4E8C1853680F0A0
:101FB0008C3609F410C28D3608F414C1843709F444
:101FC000ADC1863709F014C181E08093D20310C1FE
:101FD000813609F493C1823608F413C1823609F4BC
:101FE00008C2833609F004C18091DF039091E003B9
:101FF000892B09F036C20091DA031091DB03F80156
:102000009081992309F023C2D8018C912AE0829F04
:10201000C00111249093E0038093DF03E9C0809115
:102020000C07803709F4F7C1813708F04DC08D36B1
:1020300021F18E3609F4ACC08B3409F0B2CF009197
:10204000DA031091DB03D8018D919C9190938D045C
:1020500080938C04845E9D4F20918E0430918F0478
:10206000821B930B68E671E00E948C61845B904058
:10207000909391048093900494CF80910B018823D6
:10208000E1F3E091DA03F091DB038081813009F420
:1020900024C219828DB79EB707970FB6F8949EBFDA
:1020A0000FBE8DBFEDB7FEB731968DE4ADB7BEB7AD
:1020B00011968C9381E081838283CE010196948373
:1020C000838381E090E081C0833709F4B9C084370D
:1020D00009F4A5C1813709F064CF0091DA031091AA
:1020E000DB03D8018C918F3F09F4EEC1D8018C91AC
:1020F000882309F0DEC181E08C930091DA0310910E
:10210000DB0350E6E52E58E0F52ED8018C91B7019F
:102110004DE50E948B0480910B018823E1F3E0914F
:10212000DA03F091DB03808189838BE48A83EDB746
:10213000FEB73F970FB6F894FEBF0FBEEDBF3196C6
:1021400081E5ADB7BEB711968C9381E0818383E0C2
:102150008283CE0101969483838321E030E036832D
:102160002583CE0102969087878332872187F48664
:10217000E3868DE590E0968785870E94B10BEDB7E9
:10218000FEB73F960FB6F894FEBF0FBEEDBF09CF66
:1021900080910B018823E1F38DB79EB707970FB6A7
:1021A000F8949EBF0FBE8DBFEDB7FEB731968EE49B
:1021B000ADB7BEB711968C9381E08183828380E5B1
:1021C00095E0948383838DE490E0968385830E94D9
:1021D000B10BEDB7FEB737960FB6F894FEBF0FBE42
:1021E000EDBFDFCE873609F4F2C0883609F4DAC0D5
:1021F0001092D6031092DB031092DA031092DC03E4
:10220000C1CE8B34A9F7E091DA03F091DB03808132
:10221000918190938D0480938C04845E9D4F2091D6
:102220008E0430918F04821B930B68E671E00E944C
:102230008C61845B90409093910480939004D8CFFC
:102240000091DA031091DB03D8018C918150853025
:1022500020F411968C918B3491F0198280910B01AE
:102260008823E1F38DB79EB707970FB6F8949EBF0A
:102270000FBE8DBFEDB7FEB7319683E517CFA0E651
:10228000B8E0F80132968DE501900D928150E1F7AA
:10229000F801808160E678E04DE50E9436046091A7
:1022A0008D0870E080E090E024EC39E040E050E000
:1022B0000E944D616093A1037093A2038093A303D6
:1022C0009093A40360918E0870E080E090E00E94FB
:1022D0004D616093A5037093A6038093A703909329
:1022E000A803E091DA03F091DB0380810E94E6030A
:1022F0000E94CB0389830E94453EB0CFE091DA0370
:10230000F091DB03808180930C01803218F08FE123
:1023100080930C018FEF80930D016ACF8091D903D8
:10232000853108F4A3C0A5EEB6E08091DA03909160
:10233000DB039C01F90180E101900D928150E1F7EE
:1023400080910B018823E1F300D00F92EDB7FEB727
:10235000319684E5ADB7BEB711968C9380910E018E
:10236000818312820E94B10B8AEF8093DE038FEF8C
:1023700080930D010F900F900F903ACFE091DA0308
:10238000F091DB0380812AE0829FC00111249093A9
:10239000100180930F01892B09F42ACF81E08093EB
:1023A000D10326CF8FEF80930D01E091DA03F091F6
:1023B000DB03808190913004892B80933004882343
:1023C00011F01092D40381E08093D00311CF81E00B
:1023D0008093CE030DCF8FEF80930D01E091DA0350
:1023E000F091DB03808180932F0481E08093CF0301
:1023F000FFCEADEFB6E08091DA039091DB039C0154
:10240000F9018BE001900D928150E1F78091060770
:102410008093E2077FCF81E08093D303C2CD809188
:10242000D9038531A0F1A5EEB6E08091DA03909151
:10243000DB039C01F90180E101900D928150E1F7ED
:1024400080EF8093DE038FEF80930D01AACD8AE0A9
:10245000989FC00111240E94F5169093AC058093BB
:10246000AB050091DA031091DB03CECDE091DA03E6
:10247000F091DB0380819181A281B3818093E50695
:102480009093E606A093E706B093E80659CF009133
:10249000DA031091DB03F80180819181A281B3817D
:1024A0008093E5069093E606A093E706B093E806CE
:1024B000C7CF863008F425CE85E0F80180830091EF
:1024C000DA031091DB031DCE0E94CB03F801808359
:1024D0000091DA031091DB0309CEA0E5B5E08DE4AD
:1024E00001900D928150E1F788EE93E060E575E090
:1024F0004DE450E022E939E00E94E15F81E0898308
:10250000C9CD982F8091E307813021F0892F0E9457
:10251000650B089580912E04E82FF0E0EE5CFC4FEF
:1025200090838F5F80932E0481E008951F93182F6E
:10253000181634F480E30E94811211501116D4F35E
:102540001F9108951F93182F181634F480E20E94EB
:10255000811211501116D4F31F910895EF92FF923A
:102560000F931F93CF93DF937C018B01611571054E
:1025700069F0C0E0D0E0F701EC0FFD1FE4918E2F71
:102580000E9481122196C017D107A9F7DF91CF9140
:102590001F910F91FF90EF9008950F931F93CF938A
:1025A000DF938C01EB016115710539F0F801819120
:1025B0008F010E9481122197C9F7DF91CF911F915E
:1025C0000F9108952F923F924F925F926F927F9258
:1025D0008F929F92AF92BF92CF92DF92EF92FF9233
:1025E0000F931F93DF93CF93CDB7DEB7EA970FB664
:1025F000F894DEBF0FBECDBF61962FAD6197629696
:102600003FAD629760968FAD60978093E30742E598
:10261000A42EB12CAC0EBD1EC9018C0166247724FA
:1026200043019E01245D3F4F3AAF29AFF801F4907A
:10263000FF20A9F0F5E2FF1691F0680103C0F5E272
:10264000FF1639F00894C11CD11CF601F490FF204C
:10265000B1F7B601601B710B09F075C08601FF2050
:1026600009F495C20F5F1F4F1982EE2455244424AC
:102670004A94F8010F5F1F4FF490AE2DB0E0A170A7
:10268000B07025E7F21609F446C08F2D80628837B6
:1026900009F441C06501F0E2FF1609F44DC023E2E0
:1026A000F21609F495C04AE2F41609F495C05DE209
:1026B000F51609F4A0C0FBE2FF1609F441C02EE2B2
:1026C000F21609F444C0E0E3FE1609F496C08F2D1B
:1026D0008153893008F097C020E030E0C901880FAD
:1026E000991F880F991F880F991F220F331F280FDA
:1026F000391F2F0D311D20533040F8010F5F1F4F40
:10270000F4908F2D80538A3048F3522E560125E7DE
:10271000F21609F0BACF109709F445C094E0C92E1B
:10272000D12CCA0CDB1CF501608071808280938003
:10273000F0E2FF1609F0B3CF8981882309F046C083
:10274000F982560196CFC8010E94AE1287CFF801D8
:102750000F5F1F4F94919A3209F45FC0892F805305
:102760008A3080F5692F20E030E0C901880F991F79
:10277000880F991F880F991F220F331F280F391FA9
:10278000260F311D20533040F8010F5F1F4F649119
:10279000862F80538A3048F3A90137FD10C0442E9C
:1027A000F62E5601B4CF82E0C82ED12CCA0CDB1C09
:1027B000F501808191813C01882499246CCF4FEFF1
:1027C0005FEFEDCFF92E44245601A1CF560151CF32
:1027D00038E0E32A56014DCFA2E0AA2EB12CAC0C72
:1027E000BD1CD6015C9057FE44CF5194B0E1EB2A5A
:1027F000EFEDEE223ECF5601F9CFE4FCE7CFF0E259
:10280000EF2A560136CF28E6F216B9F04CE6F41658
:10281000C1F451E0E52A56012CCFF2E0AF2EB12CE5
:10282000AC0CBD1CD6014D915C9157FD02C0442EED
:1028300020CF4FEF5FEF442E1CCF34E0E32A560148
:1028400018CF8F2DF60193E6F91609F405C18434EB
:1028500009F472C0843609F471C0893609F46EC077
:102860008F3409F47AC18F3609F474C1803709F4C2
:1028700079C1B3E7FB1609F430C155E5F51609F443
:10288000D4C185E7F81609F4CCC1E8E5FE1609F4D1
:10289000F8C0F8E7FF1609F4F4C0FF2009F477C187
:1028A000FC8219822E2D30E03DAB2CAB5601EE247C
:1028B00034E0232E312C2C0E3D1E81E091E0E0E02F
:1028C00021E0C22ED12C2981222381F18F5F482E55
:1028D0004E0E8CA99DA98073907098AF8FAB892BF9
:1028E00029F4852D84190E94A21229812223B9F48A
:1028F0009CA996FD8CC1EFA9F8ADB09709F482C1EF
:102900008E2D0E949612C101B6010E94CD12FCA923
:10291000F4FF8CCE852D84190E94A21287CECE01A1
:10292000019661E070E00E94CD12E5CF5CA956FFF0
:10293000CECF892F8E5FCBCFB1E0EB2AE0FE54C122
:10294000B4E0AB2EB12CAC0CBD1CF60160807180E4
:102950008280938097FC3BC1BAE0BEAB47FC02C0CB
:102960005FEDE5227CE2272E312C2C0E3D1E6114FA
:1029700071048104910409F452C09EA9892F90E04A
:10298000A0E0B0E088AB99ABAAABBBAB6CE2C62EC3
:10299000D12CCC0EDD1E6CA67DA68EA69FA62AC0CD
:1029A00050E3352E360ED6013E926D016CA57DA505
:1029B0008EA59FA528A939A94AA95BA90E949F6154
:1029C000B901FA01C901DA013C014D012CA53DA56F
:1029D0004EA55FA588A999A9AAA9BBA92817390757
:1029E0004A075B0708F440C0CB01DF018CA79DA715
:1029F000AEA7BFA76CA57DA58EA59FA528A939A9BF
:102A00004AA95BA90E949F616A3050F247E5342EC3
:102A1000360E48E5F41639F65FED3522C4CF442072
:102A200089F4AE2DB0E0BDABACAB80E090E0442DBE
:102A3000E42EE91AE7FCC4C0EE2DC82EDD24C7FC45
:102A4000D09441CF3EA9232F30E040E050E028ABA6
:102A500039AB4AAB5BAB9ACFA2E0B0E0CA0EDB1E4B
:102A600080818C8319821ECF9EA99830D1F0AE2D23
:102A7000B0E0BDABACABB9ADBC198B2F9B2F160131
:102A8000D6CFE3FE1AC06114710481049104A9F049
:102A900020E4E22A8F2D30E13EAB1982F82E560158
:102AA0005DCFEE2DF0E0FDABECABE3FC0AC0F9AD81
:102AB000FC198F2F9F2F1601BACF8F2D40E14EABFF
:102AC000ECCF20E3321609F45CC0F60140E34293F8
:102AD00089AD8E1B982F1F01AACFF601208031806F
:102AE0002114310489F4F8E2FC832EE62D8335E7C6
:102AF0003E838CE68F83888789E289871A86F4E093
:102B00002F2E312C2C0E3D1E47FC1CC0442D55276A
:102B100047FD5095C10160E070E00E94B85F0097EA
:102B200019F0821948160CF4842DE2E0AE2EB12C77
:102B3000AC0CBD1C1982982F4E2D50E05DAB4CABF8
:102B400040E076CFF10101900020E9F731978E2F18
:102B50008219EBCF28E02EABA0CF31E0E32A48E08A
:102B60004EAB9BCF82E090E0C80ED91E8081918150
:102B70003C018824992490E4E92A88E7A0E1AEABDF
:102B80008CCF39AD3C19832F932F160150CFEA9685
:102B90000FB6F894DEBF0FBECDBFCF91DF911F916E
:102BA0000F91FF90EF90DF90CF90BF90AF909F90EC
:102BB0008F907F906F905F904F903F902F900895EF
:102BC000C82EDD24C7FCD094EE24E0E07CCE9094A7
:102BD000809470946094611C711C811C911CEDE2C6
:102BE000E983FAE0FEABBACEA2E0AA2EB12CAC0C7F
:102BF000BD1CD6018D919C913C01882477FC80946A
:102C0000982CA8CE852D84190E94961279CEA0E327
:102C1000AA83FB82CE01029662E070E00E94CD1290
:102C20006ACE8F2D9AE09EAB38CFA1E0EA2ABAE0B7
:102C3000BEAB33CF1F920F920FB60F9211242F937A
:102C40003F935F936F937F938F939F93AF93BF93C4
:102C50008091F003882329F08091F00381508093C4
:102C6000F0038091FE0381508093FE038F5FA9F4EF
:102C700089E08093FE03809117038F5F81708093BA
:102C80001703882309F48FC08091E9039091EA0328
:102C900001969093EA038093E9038091EE0390916B
:102CA000EF03029708F483C08091EE039091EF0345
:102CB00001979093EF038093EE038091EE03909140
:102CC000EF03209111033091120382239323892B68
:102CD00009F063C0809108018A3009F473C04798F5
:102CE0008091680883FF4BC034996EC08091EC03DB
:102CF0009091ED03892B49F18091EC039091ED03C4
:102D00008A56914010F58091EC039091ED0320914B
:102D1000EC033091ED0369E270E00E947861260FC8
:102D2000371F3093ED032093EC038091EC039091D7
:102D3000ED030B9708F454C08091EC039091ED03E0
:102D40000A9790938D0480938C0480918C049091C9
:102D50008D04845E9D4F20918E0430918F04821BE0
:102D6000930B68E671E00E948C61845B90409093C5
:102D70009104809390041092ED031092EC03BF91A4
:102D8000AF919F918F917F916F915F913F912F9123
:102D90000F900FBE0F901F901895809108018A30F8
:102DA000E9F0479A9DCF81E08093EB036DCF8FEFE1
:102DB0009FEF9093120380931103809108018A3052
:102DC00009F08DCF5A988CCF8091EC039091ED0350
:102DD00001969093ED038093EC03D1CF5A9A80CF64
:102DE00010928D0410928C04B0CF2091E9033091A1
:102DF000EA032F5F3F4F280F391FC9010895209123
:102E0000E9033091EA03821B930B80709078892F3D
:102E1000869508952091E9033091EA032F5F3F4F93
:102E2000280F391F8091E9039091EA03A901481BFB
:102E3000590BCA0180709078892F869599F308956F
:102E40002091E9033091EA032F5F3F4F280F391F8C
:102E50004FEC8091E9039091EA03B901681B790B6B
:102E6000CB0180709078892F869549F48091270353
:102E7000882379F31092270340937A00EACF0895CC
:102E80009FB7F894579A5F983E9A469AA0EBB0E0A5
:102E90008C918F708C938C9183608C93E1EBF0E03C
:102EA00080818B73808380818B6080831092B200DD
:102EB0008FEF8093B3008C9180688C93E0E7F0E013
:102EC00080818A7F80838081826080839FBF089514
:102ED0008091E9039091EA030B969093000480930C
:102EE000FF0382E085BD83EA84BD17BC88E788BD07
:102EF00086E086BDEEE6F0E0808181608083089503
:102F00001F920F920FB60F921124CF92DF92EF9281
:102F1000FF920F931F932F933F934F935F936F9362
:102F20007F938F939F93AF93BF93EF93FF93809182
:102F30000801843108F0BDC08091BE0487FDB9C08E
:102F40008091FD03882309F0B8C08091B00086FF0E
:102F500064C18091B0008F7B8093B0008091B503F5
:102F6000482F50E0440F551F440F551F2091150363
:102F700030911603C901880F991F820F931F480FC4
:102F8000591F57FD06C3CA01959587959595879555
:102F900090931603809315039093F5038093F403A5
:102FA0008091AC0880FD78C1C090F403D090F50307
:102FB000E0908308FF2400E010E0609150047091DD
:102FC0005104809152049091530420E830E040E095
:102FD00050E00E94C161C801B7010E944D61660FB7
:102FE000771F881F991F660F771F881F991F20E082
:102FF00031E040E050E00E94C161C21AD30AD09291
:10300000F503C092F40380918408282F30E0220F4A
:10301000331F220F331F8091F4039091F503821721
:1030200093077CF080918508282F30E0220F331F12
:10303000220F331F8091F4039091F503281739076D
:1030400024F43093F5032093F4032091F40330919A
:10305000F50327553E4F3093FC032093FB038091EB
:10306000F4039091F50397FD92C2959587959595F8
:1030700087959093F5038093F4038091F4039091E6
:10308000F5039093CB078093CA0745E02D3D3407A5
:1030900008F453C18CED95E09093FC038093FB03FF
:1030A0004091FB035091FC035093FA034093F903C2
:1030B0005CC08091FD03882369F14091FB0350912E
:1030C000FC0381E04F37580708F057C04F3F5105C8
:1030D00011F008F05CC04093B3001092FC03109212
:1030E000FB031092FD03FF91EF91BF91AF919F9170
:1030F0008F917F916F915F914F913F912F911F9190
:103100000F91FF90EF90DF90CF900F900FBE0F9038
:103110001F9018958091B00086FF49C08091B00043
:103120008F7B8093B0008091F803882309F08DC0D5
:103130008091860890E02DED36E0A901849F9001F2
:10314000859F300D949F300D11248091F90390914B
:10315000FA03281B390B3093FC032093FB031092D6
:10316000FA031092F903469AA90181E08093FD03C6
:1031700081E04F37580708F4A9CF8FEF8093B30051
:103180004F5F50405093FC034093FB03ACCF9A0138
:103190002F5F30402F373105C0F580E88093B300B2
:1031A000405850405093FC034093FB039CCF8091C8
:1031B000B00080648093B0008CEB90E09093FC03AF
:1031C0008093FB038091F9039091FA0384549F4FFD
:1031D0009093FA038093F9038091F103882329F0F7
:1031E00080919F04853B08F087C08091F8038F5F32
:1031F0008093F80390918608981710F41092F803C2
:103200004091FB035091FC03B0CF8FEF8093B3004C
:103210003093FC032093FB0366CF8091B000806461
:103220008093B0008091860890E02DED36E0829F7B
:10323000A001839F500D929F500D11248091F9039E
:103240009091FA03481B590B90CF29EA33E0309351
:10325000FC032093FB03823009F47AC0833009F425
:103260004DC0813009F4FBC04091FB035091FC0339
:1032700085E04D3D580708F458C04CED55E04C5BD7
:1032800050408091F9039091FA03840F951F909319
:10329000FA038093F90369CFC090F403D090F5034B
:1032A000E0908308FF2400E010E0609150047091EA
:1032B0005104809152049091530420E830E040E0A2
:1032C00050E00E94C161C801B7010E944D61660FC4
:1032D000771F881F991F660F771F881F991F20E08F
:1032E00031E040E050E00E94C161C20ED31ED09296
:1032F000F503C092F40387CE469877CFE091660835
:10330000F0E0EE0FFF1FE25DF74F80819181805E5C
:103310009F4F0CF05DC187E791E09093FC03809391
:10332000FB034091FB035091FC0381E047375807B2
:1033300008F0A5CF47E751E0A2CF2757314008F06A
:10334000AFCE87E791E09093FC038093FB03A8CE78
:103350008091BD04882309F01FC1809113039091CF
:1033600014039C01220F331F280F391F205C3E4F8E
:1033700037FD91C1359527953595279530931403E1
:103380002093130380911303909114039093F703F8
:103390008093F6038091BE0486FF4FC10091F6032F
:1033A0001091F703609158047091590480915A0468
:1033B00090915B0420E830E040E050E00E94C16161
:1033C000CA01B90128EC30E040E050E00E944D61B4
:1033D00020E031E040E050E00E94C161020F131F85
:1033E0001093F7030093F60380918408282F30E0B0
:1033F000220F331F220F331F8091F6039091F703A2
:10340000821793077CF080918508282F30E0220FE7
:10341000331F220F331F8091F6039091F703281773
:10342000390724F43093F7032093F6038091F603D1
:103430009091F70387559E4F9093FC038093FB0375
:103440008091F6039091F70397FD1EC1959587959E
:10345000959587959093F7038093F60305CF809118
:10346000B503482F50E0440F551F440F551F2091BE
:10347000150330911603C901880F991F820F931FFE
:10348000480F591F57FD04C1CA0195958795959519
:10349000879590931603809315039093F50380937B
:1034A000F4038091AC0880FF98C0C090F403D090E2
:1034B000F503E0908308FF2400E010E060915004E1
:1034C00070915104809152049091530420E830E0AF
:1034D00040E050E00E94C161C801B7010E944D6107
:1034E000660F771F881F991F660F771F881F991F08
:1034F00020E031E040E050E00E94C161C20ED31EE6
:10350000D092F503C092F40380918408282F30E014
:10351000220F331F220F331F8091F4039091F50384
:10352000821793077CF080918508282F30E0220FC6
:10353000331F220F331F8091F4039091F503281756
:10354000390724F43093F5032093F4038091F403B6
:103550009091F50387559E4F9093FC038093FB0356
:103560008091F4039091F50397FD90C09595879510
:10357000959587959093F5038093F4038091F403D8
:103580009091F5039093CB078093CA076DCE039675
:103590006CCD4D5F5F4FF7CC482F50E0440F551F67
:1035A000440F551F2091130330911403C901880F54
:1035B000991F820F931F480F591F57FD6FC05595D4
:1035C0004795559547955093140340931303DACECE
:1035D0003093FC032093FB03A4CEC090F403D0905F
:1035E000F503E0908308FF2400E010E060915004B0
:1035F00070915104809152049091530420E830E07E
:1036000040E050E00E94C161C801B7010E944D61D5
:10361000660F771F881F991F660F771F881F991FD6
:1036200020E031E040E050E00E94C161C21AD30ABC
:10363000D092F503C092F40367CF0091F603109186
:10364000F703609158047091590480915A04909145
:103650005B0420E830E040E050E00E94C161CA0114
:10366000B90120EA30E040E050E00E944D6120E0E6
:1036700031E040E050E00E94C161021B130B109347
:10368000F7030093F603B0CE0396E0CE03966ECF19
:103690004D5F5F4FF9CE2D5F3F4F6CCE4D5F5F4F5B
:1036A0008ECF10927C008FEC80937A0008951F9249
:1036B0000F920FB60F921124DF92EF92FF920F93A9
:1036C0001F932F933F934F935F936F937F938F93AA
:1036D0009F93AF93BF93CF93DF93EF93FF93D090DC
:1036E0002A048D2DD394D0922A04E82FF0E0E23101
:1036F000F105F8F010922A0482E080932B04809365
:103700007C00FF91EF91DF91CF91BF91AF919F919D
:103710008F917F916F915F914F913F912F911F9169
:103720000F91FF90EF90DF900F900FBE0F901F90C2
:103730001895E25CFF4FEE0FFF1F0590F491E02D0E
:10374000099480917800909179002091240430911F
:103750002504280F391F309325042093240481E089
:1037600080932B0480912B0480937C00DD2049F210
:103770008FEC80937A00C5CF10922A0481E0809369
:1037800027038091170490911804019690931804D0
:1037900080931704DD242091780030917900809186
:1037A000F4079091F507820F931F9093F50780938C
:1037B000F4078091EC078F5F8093EC078091EC0712
:1037C000853008F4B5C08091F4079091F50797FD16
:1037D00078C3959587959093F5078093F40780912A
:1037E00078009091790090932303809322031092A4
:1037F000EC076091150470911604809114049927C8
:1038000087FD9095D82FCC27C81BD90B2091E807AE
:103810003091E9078091F4079091F5074091A90450
:103820005091AA04281B390B241B350B2C0F3D1F6C
:103830008091AB0390E0289FA001299F500D389FF5
:10384000500D11248FE190E09C01629FC001639FA5
:10385000900D729F900D1124480F591F57FD2EC3D4
:103860005595479555954795559547955595479540
:103870005595479550931604409315046091F407AD
:103880007091F507E0901E03F0901F030091200354
:1038900010912103882777FD8095982FA801970123
:1038A000220F331F441F551F220F331F441F551F64
:1038B000220F331F441F551F2E193F09400B510B78
:1038C000620F731F841F951F6C5F7F4F8F4F9F4F39
:1038D00028E030E040E050E00E94C161C901DA0117
:1038E00080931E0390931F03A0932003B0932103A2
:1038F0002091E8073091E90780911E0390911F0302
:10390000A0912003B0912103C20FD31FC81BD90B74
:10391000D093AA04C093A9048091F4079091F5076D
:1039200097FDCAC2959587959093F5078093F40704
:1039300082E080932B0416CF60917800709179001B
:10394000E0904A04F0904B0400914C0410914D0417
:10395000882777FD8095982F0E949960A80197018C
:103960000E94FD5F0E9466607093120460931104D0
:10397000809111049091120402970CF44FC260914F
:103980004A0470914B0480914C0490914D0420E0C6
:1039900030E84BE354E40E94626088239CF5609118
:1039A0004A0470914B0480914C0490914D042AE09C
:1039B00037ED43EA5CE30E94FE5F60934A04709334
:1039C0004B0480934C0490934D048091C9049091D2
:1039D000CA04845F9140B0F460914A0470914B0432
:1039E00080914C0490914D042DEC3CEC4CEC5DE34B
:1039F0000E94FE5F60934A0470934B0480934C04D2
:103A000090934D0481E0809313048091780090910D
:103A100079009093E7078093E607809111049091D5
:103A20001204209188043091890440918A045091B5
:103A30008B04AA2797FDA095BA2F820F931FA41F6E
:103A4000B51F8093880490938904A0938A04B0934F
:103A50008B04609188047091890480918A0490910C
:103A60008B04E0908804F090890400918A041091FE
:103A70008B0420E034E040E050E00E94C161E21A93
:103A8000F30A040B150BE0928804F092890400936A
:103A90008A0410938B0483E080932B0463CE80917F
:103AA0007800909179002091260430912704280F06
:103AB000391F309327042093260484E080932B043D
:103AC00051CE409118035091190380917800909144
:103AD00079009A01220F331F240F351F63E070E035
:103AE0000E947861260F371F3695279536952795C2
:103AF000309319032093180385E080932B0432CE72
:103B00008091780090917900909329048093280403
:103B100086E080932B0426CE2091780030917900A6
:103B20008091460490914704821B930B9093E50784
:103B30008093E4078091E4079091E50790931F0438
:103B400080931E0487E080932B040CCE8091780034
:103B5000909179002091440430914504821B930B8D
:103B60009093F0078093EF078091EF079091F00713
:103B700090931D0480931C0482E080932B04F2CD6B
:103B8000209178003091790080912604909127044B
:103B9000820F931F909327048093260410922B0486
:103BA000E1CD809108018A3009F418C1843109F40B
:103BB0008AC18091780090917900209128043091F9
:103BC0002904820F931F90930C0480930B0486E0CA
:103BD00080932B04C7CD209178003091790080919B
:103BE000460490914704821B930B9093E5078093C2
:103BF000E4078091E4079091E50720911E0430913D
:103C00001F04820F931F90930E0480930D0487E08E
:103C100080932B04A7CD809178009091790020911A
:103C2000440430914504821B930B9093F0078093DA
:103C3000EF078091EF079091F00720911C043091DD
:103C40001D04820F931F9093100480930F0482E051
:103C500080932B0487CD209178003091790080915A
:103C6000240490912504280F391F809108018A307F
:103C700009F4CDC0220F331F220F331F30932504C8
:103C8000209324042091240430912504C90137FD98
:103C900039C1959587959595879595958795909335
:103CA0000804809307048091220490912304820FDA
:103CB000931F97FD25C19595879590932304809335
:103CC000220420913A0430913B04821B930B909381
:103CD0001B0380931A0380910104909102042091A8
:103CE0001A0330911B03280F391F37FD06C1359584
:103CF0002795309302042093010481E080932B04E4
:103D000031CD2091780030917900809126049091F6
:103D10002704280F391F809108018A3009F470C0E8
:103D2000220F331F220F331F3093270420932604C2
:103D30002091260430912704C90137FDD9C09595FB
:103D40008795959587959595879590930A04809387
:103D500009048091200490912104820F931F97FD04
:103D6000C5C0959587959093210480932004209158
:103D70003C0430913D04821B930B90931D03809370
:103D80001C03809103049091040420911C03309142
:103D90001D03280F391F37FDADC03595279530938A
:103DA00004042093030483E080932B04DBCC8091F4
:103DB000780090917900909325048093240481E009
:103DC00080932B04CFCC80917800909179009093D0
:103DD00027048093260410922B04C4CC8091780091
:103DE0009091790001962091280430912904820F46
:103DF000931F9695879590930C0480930B04E7CEC0
:103E0000220F331F309327042093260491CF220FD3
:103E1000331F309325042093240434CF8091110460
:103E2000909112048F5F9F4F0CF0ECCD60914A048B
:103E300070914B0480914C0490914D0420E030E847
:103E400049E054E40E94496118160CF0DBCD609102
:103E50004A0470914B0480914C0490914D042AE0E7
:103E600037ED43EA5CE30E94FD5F60934A04709380
:103E70004B0480934C0490934D048091C90490911D
:103E8000CA04845F914008F0BDCD60914A047091EE
:103E90004B0480914C0490914D042DEC3CEC4CEC87
:103EA0005DE30E94FD5F60934A0470934B0480932E
:103EB0004C0490934D04A6CD019634CD415E5F4FE6
:103EC000CFCC019686CC80917800909179002FEF2D
:103ED00037E0281B390B8091280490912904281B76
:103EE000390B30930C0420930B0471CE019639CF1B
:103EF000079625CF2F5F3F4F50CF2F5F3F4FF7CE15
:103F00000196D9CE0796C5CE9F92AF92BF92CF921F
:103F1000DF92EF92FF920F931F93CF93DF93109254
:103F2000190410921A0410921B0480ED97E00E946D
:103F3000F516EC010CE8FF24F394B8E0CB2EA5EFC6
:103F4000EA2EFAE0DF2EE1EBAE2EE2E0BE2E7FECB1
:103F5000972E80910704909108048C5F93400CF099
:103F600099C08091240381508093240310E08091B4
:103F7000090490910A048C5F93400CF07EC08091FC
:103F8000250381508093250380910B0490910C04AC
:103F90008C5F93400CF064C0809126038150809325
:103FA0002603C09231040E94122A809124038A3091
:103FB00008F04EC0F0921904D0922403809125039A
:103FC0008A3008F03EC0F0921A04D0922503809106
:103FD00026038A3078F5F0921B04D0922603809154
:103FE0003104882389F0CE010E94FF168823B9F39B
:103FF00000D00F92EDB7FEB71182B382A2820E9469
:10400000E2120F900F900F901092EC0790927A00AE
:104010008091EC078823E1F30A3008F444C0015092
:1040200009F448C0133009F094CF0B3008F491CF55
:1040300009E08FCF863F98F2F0921B04E0922603AE
:10404000CECF863F20F2F0921A04E0922503BFCF34
:10405000863F08F4B3CFF0921904E0922403AECF68
:1040600080910B0490910C04875094409CF18091B6
:1040700026038F5F8093260394CF8091090490914B
:104080000A048750944044F1809125038F5F809308
:1040900025037ACF809107049091080487509440BB
:1040A000ECF411E064CF8AE090E00E942017015008
:1040B00009F0B8CF86E490E00E942017DF91CF91FD
:1040C0001F910F91FF90EF90DF90CF90BF90AF9036
:1040D0009F9008951F5F65CF1F5F56CF8091240387
:1040E0008F5F8093240310E042CFEF92FF920F93F3
:1040F0001F93CF93DF93F999FECF13E0E12E10E0E9
:10410000F12EF2BCE1BCF89A80B5C82FD0E0C531E1
:10411000D10508F02A97C7BD1092140484E690E0F8
:104120000E9420178091220390912303825593408F
:1041300008F03AC0C0E0D0E008EE12E004C02196DA
:10414000CA3FD105C0F4C7BD82E390E00E942017AA
:1041500000D00F92EDB7FEB71182138302830E9445
:10416000E21280912203909123030F900F900F9001
:104170008255934020F78C2FF999FECF1FBAF2BCDD
:10418000E1BC80BD0FB6F894FA9AF99A0FBE8093FD
:10419000F1078CE291E00E942017DF91CF911F91EF
:1041A0000F91FF90EF900895CA3FD10520F708EED8
:1041B00012E0C9CFE2E3F3E080E2819393E0E238DA
:1041C000F907D9F70895FF920F931F93CF93DF93C9
:1041D0003091820380912F04381710F430932F040C
:1041E0008091300490E080FF08C020912F042223AA
:1041F00009F495C1215020932F0481FF08C020911C
:104200002F04321709F48EC12F5F20932F0483707F
:104210009070039711F410922F04E2E3F3E080E230
:10422000819323E0E238F207D9F720912F042A3056
:1042300008F097C081E180932E0400D000D00F9247
:10424000EDB7FEB7319681E0ADB7BEB711968C934E
:1042500081EE96E092838183238314820E94E2128E
:104260000F900F900F900F900F9010912F04163019
:1042700009F445C5173008F485C01A3009F461C443
:104280001B3008F052C1183009F4ECC5193008F49D
:10429000B5C510922E0400D000D00F92EDB7FEB736
:1042A000319611E0ADB7BEB711961C938FE194E043
:1042B000928381838091970490919804948383835F
:1042C0000E94E21284E180932E04EDB7FEB731968E
:1042D000ADB7BEB711961C9383E194E092838183BE
:1042E0008091990490919A04948383830E94E212AE
:1042F00088E280932E04EDB7FEB73196ADB7BEB716
:1043000011961C9387E094E09283818380919B04B3
:1043100090919C04948383830E94E2128CE38093A7
:104320002E04EDB7FEB73196ADB7BEB711961C930C
:104330008BEF93E09283818380919D0490919E0402
:10434000948383830E94E2120F900F900F900F903E
:104350000F9010923004DF91CF911F910F91FF9039
:10436000089580E180932E0400D000D00F92EDB725
:10437000FEB7319681E0ADB7BEB711968C938CED48
:1043800096E068CF123009F43EC4133008F4A6C199
:10439000143009F4C4C2153008F442C210922E043D
:1043A00000D00F9211E0ADB7BEB711961C931197D4
:1043B00081E695E013969C938E9312970E94E212E9
:1043C000809108010F900F900F908A3009F47BC7FD
:1043D0008B3009F4B8C6843109F4B5C68D3009F0C4
:1043E000B8CF84E180932E0460913A0470913B042D
:1043F00040910704509108042DB73EB72950304032
:104400000FB6F8943EBF0FBE2DBFCDB7DEB72196D5
:1044100081E0ADB7BEB711968C9387EE94E09A8396
:1044200089839B01C90137FDF5C7959587959595BA
:10443000879595958795481B590B5C834B839B010A
:1044400077FDE5C7359527953595279535952795BA
:10445000359527953E832D83809124038F8318867D
:104460000E94E21288E280932E0460913C047091D5
:104470003D044091090450910A0481E0888383ED52
:1044800094E09A8389839B01C90137FDBEC7959546
:1044900087959595879595958795481B590B5C83CE
:1044A0004B839B0177FDAEC73595279535952795AD
:1044B00035952795359527953E832D838091250346
:1044C0008F8318860E94E2128CE380932E04409121
:1044D0003E0450913F0420910B0430910C0481E084
:1044E00088838FEB94E09A838983CA01821B930BA4
:1044F0009C838B8357FD79C7559547955E834D8384
:10450000809126038F8318860E94E212EDB7FEB7D2
:1045100039960FB6F894FEBF0FBEEDBF1ACF309399
:104520002F046BCE10922F0472CE1C3009F456C5A6
:104530001C3008F4EEC41D3009F0D5C010922E04D2
:1045400000D00F9211E0ADB7BEB711961C93119732
:104550008BE293E013969C938E9312970E94E21243
:1045600084E180932E04EDB7FEB738970FB6F89428
:10457000FEBF0FBEEDBF3196ADB7BEB711961C930F
:1045800087E193E0928381838091220890E08D9669
:10459000948383838091230890E08D96968385830E
:1045A0008091240890E08D969087878380912508DC
:1045B00090E08D96928781870E94E21288E2809334
:1045C0002E04EDB7FEB73196ADB7BEB711961C936A
:1045D00083E093E0928381838091260890E08D961A
:1045E000948383838091270890E08D9696838583BA
:1045F0008091280890E08D96908787838091290884
:1046000090E08D96928781870E94E2128CE38093DE
:104610002E04EDB7FEB736960FB6F894FEBF0FBE68
:10462000EDBF3196ADB7BEB711961C9383EF92E004
:104630009283818380912A0890E08D96948383836E
:104640000E94E2120F900F900F900F900F908091A8
:104650002B08882389F080E480932E0400D00F92E9
:10466000EDB7FEB7118380EF92E0938382830E94BF
:10467000E2120F900F900F9080912C088823B1F0D8
:1046800084E480932E0400D00F9281E0ADB7BEB7D2
:1046900011968C9311978DEE92E013969C938E93C6
:1046A00012970E94E2120F900F900F9080912D08A8
:1046B000882309F44ECE88E480932E0400D00F9214
:1046C00081E0EDB7FEB781838AEE92E09383828327
:1046D0000E94E2120F900F900F903BCE112349F0F1
:1046E000113009F4CCC111501093820310922F04A1
:1046F00030CE10922E0400D00F9211E0EDB7FEB72D
:1047000011838CEC96E0938382830E94E21284E111
:1047100080932E04209108018DB79EB70A970FB69B
:10472000F8949EBF0FBE8DBFEDB7FEB73196ADB703
:10473000BEB711961C9387EB96E092838183822FFC
:104740006AE00E946C6183831482822F0E946C61F4
:1047500095831682108617828AE490E0928781877B
:1047600084E690E0948783870E94E21288E2809337
:104770002E04EDB7FEB73D960FB6F894FEBF0FBE00
:10478000EDBF0E94CB032DB73EB7275030400FB688
:10479000F8943EBF0FBE2DBFEDB7FEB73196ADB753
:1047A000BEB711961C9329EA36E0328321838383B6
:1047B000148281E595E0968385830E94E2128091C0
:1047C0009D0390919E03EDB7FEB737960FB6F89410
:1047D000FEBF0FBEEDBF069708F45FC5809134049D
:1047E000882309F49EC48CE380932E0400D000D06B
:1047F0000F92EDB7FEB73196ADB7BEB711961C93C9
:1048000087E896E0928381838091340483831482C5
:104810000E94E2120F900F900F900F900F9099CD81
:1048200010922E04209130083091310840913208C6
:1048300050913308EDB7FEB737970FB6F894FEBF27
:104840000FBEEDBF319611E0ADB7BEB711961C9308
:104850008FED95E092838183348323835683458350
:104860000E94E21284E180932E042091340830915A
:1048700035084091360850913708EDB7FEB73196AC
:10488000ADB7BEB711961C938FEC95E092838183F0
:1048900034832383568345830E94E21288E2809307
:1048A0002E04209138083091390840913A085091EF
:1048B0003B08EDB7FEB73196ADB7BEB711961C9366
:1048C0008FEB95E0928381833483238356834583E2
:1048D0000E94E2128CE380932E0420913C083091D8
:1048E0003D0840913E0850913F08EDB7FEB7319624
:1048F000ADB7BEB711961C938FEA95E09283818382
:1049000034832383568345830E94E212EDB7FEB7BA
:1049100037960FB6F894FEBF0FBEEDBF1ACD1092BA
:104920002E04E0916008F0E0EE0FFF1FE25DF74F0C
:1049300040815181E0916108F0E0EE0FFF1FE25DE0
:10494000F74F208131818DB79EB707970FB6F89446
:104950009EBF0FBE8DBFEDB7FEB7319611E0ADB76C
:10496000BEB711961C938FE995E09283818354839F
:104970004383368325830E94E21284E180932E04D0
:10498000E0916208F0E0EE0FFF1FE25DF74F40811B
:104990005181E0916308F0E0EE0FFF1FE25DF74FF9
:1049A00020813181EDB7FEB73196ADB7BEB7119614
:1049B0001C938FE895E092838183548343833683ED
:1049C00025830E94E21288E280932E04E09164081D
:1049D000F0E0EE0FFF1FE25DF74F40815181E09163
:1049E0006508F0E0EE0FFF1FE25DF74F2081318197
:1049F000EDB7FEB73196ADB7BEB711961C938FE7F2
:104A000095E09283818354834383368325830E9478
:104A1000E2128CE380932E04E0916608F0E0EE0F42
:104A2000FF1FE25DF74F40815181E0916708F0E0A0
:104A3000EE0FFF1FE25DF74F20813181EDB7FEB72A
:104A40003196ADB7BEB711961C938FE695E0928371
:104A5000818354834383368325830E94E212EDB71A
:104A6000FEB737960FB6F894FEBF0FBEEDBF10929B
:104A70003004DF91CF911F910F91FF9008958091A5
:104A8000680880FF2CC310922E0400D000D00F9233
:104A9000EDB7FEB73196ADB7BEB711961C9388E659
:104AA00096E0928381838091A9049091AA049483D3
:104AB00083830E94E21284E180932E04EDB7FEB757
:104AC0003196ADB7BEB711961C9389E596E09283F7
:104AD00081838091AB049091AC04948383830E9482
:104AE000E21288E280932E04209122033091230366
:104AF000EDB7FEB73196ADB7BEB711961C938AE4F9
:104B000096E092838183348323830E94E2128CE3B4
:104B100080932E04EDB7FEB73196ADB7BEB71196B0
:104B20001C938BE396E0928381838091F1078383CA
:104B300014820E94E2120F900F900F900F900F902E
:104B400008CC10922E0400D00F9211E0EDB7FEB702
:104B5000118383EF93E0938382830E94E21284E1C6
:104B600080932E0400D0EDB7FEB73196ADB7BEB737
:104B700011961C9385EE93E0928381838091B50317
:104B8000838314820E94E21288E280932E04EDB7A0
:104B9000FEB73196ADB7BEB711961C9387ED93E083
:104BA000928381838091F2039091F30394838383B2
:104BB0000E94E2128CE380932E0400D0EDB7FEB782
:104BC0003196ADB7BEB711961C9389EC93E09283F2
:104BD00081838091840883831482809185088583F2
:104BE00016820E94E212EDB7FEB737960FB6F89420
:104BF000FEBF0FBEEDBF10923004DF91CF911F9129
:104C00000F91FF90089510922E0400D00F92FF2470
:104C1000F394EDB7FEB7F1828CE196E09383828343
:104C20000E94E21284E180932E0400D000D00DB7E0
:104C30001EB70F5F1F4FADB7BEB71196FC928DE048
:104C400096E0F80192838183609150047091510441
:104C5000809152049091530420E034E040E050E011
:104C60000E94C161D80113962D933D934D935C939F
:104C700016970E94E21288E280932E040DB71EB7A9
:104C80000F5F1F4FEDB7FEB7F1828EEF95E0D801B1
:104C900012969C938E9311976091580470915904C9
:104CA00080915A0490915B0420E034E040E050E0B1
:104CB0000E94C161F80123833483458356830E9497
:104CC000E2128CE380932E040F900F90EDB7FEB7A5
:104CD0003196ADB7BEB71196FC928FEE95E09283F8
:104CE000818380918C0490918D04948383830E94AE
:104CF000E2120F900F900F900F900F902ACB10920E
:104D00002E0400D00F92FF24F394ADB7BEB71196D6
:104D1000FC92119782EB94E013969C938E931297DA
:104D20000E94E21284E180932E0420910F043091BE
:104D3000100400D000D0EDB7FEB73196ADB7BEB7C6
:104D40001196FC9283EA94E09283818334832383D7
:104D50008091440490914504968385830E94E212D9
:104D600088E280932E0420910D0430910E04EDB75B
:104D7000FEB73196ADB7BEB71196FC9284E994E0C8
:104D800092838183348323838091460490914704E6
:104D9000968385830E94E2128CE380932E046091B7
:104DA0004A0470914B0480914C0490914D040DB7CE
:104DB0001EB70F5F1F4FEDB7FEB7F18225E834E055
:104DC000D80112963C932E9311972091D9083091D7
:104DD000DA0814963C932E9313970E946660F801AC
:104DE000768365830E94E2122DB73EB7295F3F4F5D
:104DF0000FB6F8943EBF0FBE2DBFABCA84E18093BF
:104E00002E04209118033091190300D000D00F9286
:104E1000EDB7FEB7319611E0ADB7BEB711961C9352
:104E200086E794E092838183348323830E94E21295
:104E300088E280932E0420919F04EDB7FEB731964F
:104E4000ADB7BEB711961C9387E694E09283818339
:104E5000238314820E94E2120F900F900F900F9004
:104E60000F9077CA10922E0400D00F9211E0EDB788
:104E7000FEB7118388E594E0938382830E94E21257
:104E800084E180932E0400D0EDB7FEB73196ADB724
:104E9000BEB711961C9389E494E09283818380913C
:104EA000900490919104948383830E94E21288E29B
:104EB00080932E04EDB7FEB73196ADB7BEB711960D
:104EC0001C938AE394E09283818380918C04909177
:104ED0008D04948383830E94E2128CE380932E04DA
:104EE000EDB7FEB73196ADB7BEB711961C938BE206
:104EF00094E09283818380918E0490918F049483B7
:104F000083830E94E2120F900F900F900F900F90EA
:104F100020CA10922E0400D00F9211E0ADB7BEB798
:104F200011961C93119789EB93E013969C938E93A3
:104F300012970E94E21284E180932E0400D000D0E8
:104F4000EDB7FEB73196ADB7BEB711961C9389EA9F
:104F500093E09283818380910007992787FD909544
:104F60009483838380910107992787FD9095968389
:104F700085830E94E21288E280932E04EDB7FEB78B
:104F80003196ADB7BEB711961C9389E993E0928331
:104F9000818380910307838314828091020799277C
:104FA00087FD9095968385830E94E2128CE380931F
:104FB0002E04EDB7FEB73196ADB7BEB711961C9370
:104FC00089E893E09283818380910407992787FD84
:104FD0009095948383838091070701CE10922E04CD
:104FE00000D00F9211E0ADB7BEB711961C93119788
:104FF00089E793E013969C938E9312970E94E21296
:1050000084E180932E04EDB7FEB738970FB6F8947D
:10501000FEBF0FBEEDBF3196ADB7BEB711961C9364
:1050200084E693E0928381838091060883831482CF
:1050300080910708858316828091080887831086EF
:1050400080910908818712860E94E21288E280938B
:105050002E04EDB7FEB73196ADB7BEB711961C93CF
:105060008FE493E09283818380910A088383148282
:1050700080910B088583168280910C0887831086A7
:1050800080910D08818712860E94E2128CE3809342
:105090002E04EDB7FEB73196ADB7BEB711961C938F
:1050A0008AE393E09283818380910E088383148244
:1050B00080910F088583168280911008878310865F
:1050C00080911108818712860E94E212EDB7FEB727
:1050D0003B960FB6F894FEBF0FBEEDBF3AC984E110
:1050E00080932E0400D00F92EDB7FEB7118384E3B6
:1050F00096E0938382830E94E21288E280932E04DA
:10510000ADB7BEB711961C93119786E296E0139641
:105110009C938E9312970E94E2120F900F900F9023
:1051200018C98CE380932E0400D00F92EDB7FEB720
:10513000118387E796E0938382830E94E2120F90A7
:105140000F900F9006C984E180932E0460913A0479
:1051500070913B0440910704509108042DB73EB76D
:10516000295030400FB6F8943EBF0FBE2DBFCDB7CB
:10517000DEB7219681E0ADB7BEB711968C938CE176
:1051800095E09A8389839B01C90137FD0796959520
:1051900087959595879595958795481B590B5C83C1
:1051A0004B839B0177FF02C0215F3F4F35952795C9
:1051B0003595279535952795359527953E832D83EC
:1051C000CB0160E170E00E948C6197FD019695959E
:1051D000879598878F830E94E21288E280932E043D
:1051E00060913C0470913D044091090450910A047F
:1051F00081E088838AE095E09A8389839B01C901D5
:1052000037FD0796959587959595879595958795FB
:10521000481B590B5C834B839B0177FF02C0215FC6
:105220003F4F359527953595279535952795359594
:1052300027953E832D83CB0160E170E00E948C6155
:1052400097FD01969595879598878F830E94E21226
:105250008CE380932E0420913E0430913F044091D2
:105260000B0450910C040F900F90EDB7FEB73196E0
:1052700081E0ADB7BEB711968C938BEF94E092832B
:105280008183C901841B950B9483838337FF02C0FC
:105290002F5F3F4F35952795DECB8CE380932E040F
:1052A00000D00F92ADB7BEB711961C9311978CE941
:1052B00096E013969C938E9312970E94E2120F90A1
:1052C0000F900F9046C884E180932E0460913A04B9
:1052D00070913B044091070450910804EDB7FEB76C
:1052E00039970FB6F894FEBF0FBEEDBFCDB7DEB74E
:1052F0002196ADB7BEB711961C938FE495E09A83C3
:1053000089839B01C90137FD7BC09595879595954C
:10531000879595958795481B590B5C834B839B011B
:1053200077FD6BC03595279535952795359527954C
:105330003E832D83CB0168E070E00E948C619887EA
:105340008F830E94E21288E280932E0460913C04D5
:1053500070913D044091090450910A0481E08883D2
:105360008DE395E09A8389839B01C90137FD43C092
:10537000959587959595879595958795481B590B94
:105380005C834B839B0177FD33C03595279535951D
:105390002795359527953E832D83CB0168E070E0F6
:1053A0000E948C6198878F830E94E2128CE3809325
:1053B0002E0420913E0430913F0440910B04509103
:1053C0000C040F900F90EDB7FEB7319681E0ADB7AA
:1053D000BEB711968C938EE295E092838183C901CA
:1053E000841B950B9483838336CB4F5F5F4F84C8B8
:1053F000295F3F4FCACF0796BBCF295F3F4F92CF60
:10540000079683CF215F3F4F4FC8079640C8215F63
:105410003F4F18C8079609C81092B9008AE28093D6
:10542000B800089585EA8093BC00089584E98093CC
:10543000BC0008954CEB50E084E9DA018C931092A3
:1054400031042BEB30E0F90180811092320480E8C6
:105450008C931092BD001092BA001082E9EBF0E03C
:105460001082A8EBB0E01C9210828AE28C9385EA4D
:10547000DA018C931082F901108285E88C930895EB
:105480001092B9008093BB0085E88093BC0008951A
:105490008093BB0085E88093BC00089585EC8093E1
:1054A000BC00089585E88093BC0008951F920F9278
:1054B0000FB60F9211242F933F938F939F93EF93E7
:1054C000FF93809131048F5F809331048150E82FE6
:1054D000F0E0E731F10590F0109231048091BC00CA
:1054E00080688093BC00FF91EF919F918F913F91D5
:1054F0002F910F900FBE0F901F901895E05BFF4FFC
:10550000EE0FFF1F0590F491E02D09941092B90061
:1055100088E98093BB0085E88093BC00DFCF1092C0
:10552000B90080E88093BB0085E88093BC00D6CFAB
:1055300084E98093BC008AE090E090939E0380937E
:105540009D0385EA8093BC00C9CF90913204292F36
:1055500030E0F901EE0FFF1FEE0FFF1FE05BFA4F87
:1055600085851816A4F09C3018F011C09C3068F4A2
:105570009F5F292F30E0F901EE0FFF1FEE0FFF1F95
:10558000E05BFA4F858518168CF7909332049C30B7
:1055900009F4D6C0275D3F4F220F331F1092B90088
:1055A0002093BB0085E88093BC0098CF80912503B1
:1055B0001092B9008093BB0085E88093BC008ECF29
:1055C0001092B90082E18093BB0085E88093BC0013
:1055D00085CF809126031092B9008093BB0085E8A7
:1055E0008093BC007BCF809124031092B9008093FC
:1055F000BB0085E88093BC0071CF84E98093BC0038
:105600008AE090E090939E0380939D031092310472
:1056100065CF1092B90084E18093BB0085E8809348
:10562000BC005CCF8091B900803309F46AC084E982
:105630008093BC008AE090E090939E0380939D034A
:105640001092310485EA8093BC0048CF80913204E7
:10565000E82FF0E0E35FF64F90818F5F8093320494
:105660001092B9009093BB0085E88093BC0036CFC0
:105670001092B90080E18093BB0085E88093BC0064
:105680002DCF809133049091BB00E82FF0E0EA50D9
:10569000F84F90838F5F809333048C3010F010921A
:1056A000330484E98093BC001092310417CF8091B9
:1056B000BB00E0913304F0E0EE5EF74F808385E8B5
:1056C0008093BC000BCF8091B900803469F1809148
:1056D0003304E82FF0E0EE5DF74F10828F5F809388
:1056E00033048C3010F01092330484E98093BC00B2
:1056F0001092310480913504809334041092350463
:10570000EDCE80913504882361F180913204E82F39
:10571000F0E0EB5FF74F80818F5F8083882309F093
:1057200086CF8FEF808383CF80913304E82FF0E022
:10573000EE5DF74F8C5F808385EC8093BC00DACF01
:105740001092320483E08093310480913304880FF7
:105750008D5A1092B9008093BB0085E88093BC00FD
:10576000BDCE8091320480933504D1CF83EC8093F9
:105770008100EFE6F0E080818062808310923F0438
:1057800010923E0410923D0410923C0410923B048F
:1057900010923A0408951F920F920FB60F9211249F
:1057A0000F931F932F933F934F935F936F937F9329
:1057B0008F939F93AF93BF93CF93DF93EF93FF9319
:1057C00020918600309187008091380490913904AF
:1057D000281B390B809186009091870090933904A3
:1057E00080933804C9018D549440835F9A4118F521
:1057F0008091360490913704049714F0109283033B
:1058000081E090E09093370480933604FF91EF910C
:10581000DF91CF91BF91AF919F918F917F916F91C8
:105820005F914F913F912F911F910F910F900FBE5C
:105830000F901F90189500913604109137040A308C
:10584000110524F7C9018B5F9040845B914008F0FB
:1058500056C0A901425D5140E801CC0FDD1FFE0199
:10586000E25DF74F808191819A01281B390BC901B4
:1058700037FD74C0069754F480919F04883C08F06B
:1058800066C080919F04865F80939F04FE01E25D65
:10589000F74F808191819C01220F331F280F391F00
:1058A000240F351F37FD57C035952795359527951A
:1058B000CA010196821793070CF040C02150304076
:1058C00080919F04833CA0F1FE01E25DF74F80814F
:1058D0009181A901481B590BCA0163E070E00E9445
:1058E0008C61CB01880F991F860F971FFE01EC5B1F
:1058F000F74F91838083C25DD74F39832883C801D6
:10590000019690933704809336048530910549F0D1
:105910005D988630910549F05C98079721F45B9A71
:1059200075CF5D9A5C985B9871CF5C9A5B986ECFEF
:10593000FE01EC5BF74F11821082DDCF41505040E9
:10594000241735070CF0BCCF2F5F3F4FB9CF88EC41
:1059500080939F049BCF2D5F3F4FA6CF909581955D
:105960009F4F88CF81E08093600882E08093610838
:1059700083E08093620884E08093630885E08093ED
:10598000640886E08093650887E08093660888E075
:105990008093670808959C01CB0162177307B4F0E8
:1059A0006091BC04662359F06130D9F0821B930BDF
:1059B00070E00E948C61620F731FCB010895B901E2
:1059C000660F771F681B790BCB010895620F731F59
:1059D00077FD04C075956795CB0108956F5F7F4F84
:1059E000F9CFBC01621B730B77FD07C075956795F6
:1059F000C901861B970BBC01E0CF6F5F7F4FF6CFCD
:105A00002F923F924F925F926F927F928F929F92CE
:105A1000AF92BF92CF92DF92EF92FF920F931F93BC
:105A2000DF93CF93CDB7DEB7A1970FB6F894DEBF63
:105A30000FBECDBF80910B0490910C0420913E04C9
:105A400030913F04281B390B39A328A330931C093C
:105A500020931B09209101043091020437FF02C0FA
:105A60000C947E35C9019595879595958795959563
:105A700087959A8F898F209103043091040437FF12
:105A800002C00C947A35D901B595A795B595A7951F
:105A9000B595A795B88FAF8BE98DFA8DF093DC089B
:105AA000E093DB08B093D208A093D10860910F0473
:105AB00070911004882777FD8095982F26E030E0BC
:105AC00040E050E00E944D617B018C0120910A0969
:105AD00030910B09442737FD4095542FCA01B90175
:105AE000660F771F881F991F620F731F841F951FF2
:105AF0006E0D7F1D801F911F24E030E040E050E0DC
:105B00000E94C16130930B0920930A0960910D0432
:105B100070910E04882777FD8095982F26E030E05D
:105B200040E050E00E944D617B018C0120912609EC
:105B300030912709442737FD4095542FCA01B901F8
:105B4000660F771F881F991F620F731F841F951F91
:105B50006E0D7F1D801F911F24E030E040E050E07B
:105B60000E94C1613093270920932609E090110417
:105B7000F09012042091D9083091DA08442737FDBB
:105B80004095542FCA01B901660F771F881F991FCE
:105B9000620F731F841F951F0027F7FC0095102FBD
:105BA0006E0D7F1D801F911F24E030E040E050E02B
:105BB0000E94C1613093DA082093D90820910F0424
:105BC00030911004C901880F991F820F931F880F0D
:105BD000991FAA2797FDA095BA2F209160043091B4
:105BE00061044091620450916304280F391F4A1FD9
:105BF0005B1F2093600430936104409362045093D0
:105C0000630420910D0430910E04C901880F991F7F
:105C1000820F931F880F991FAA2797FDA095BA2F6F
:105C200020916404309165044091660450916704AA
:105C3000280F391F4A1F5B1F2093640430936504AB
:105C4000409366045093670420910F043091100430
:105C50008091E4089091E508820F931F9093E508E6
:105C60008093E40820910D0430910E0480911E0968
:105C700090911F09820F931F90931F0980931E0913
:105C8000809148049091490401969093490480932F
:105C90004804E090E607F090E707A0904A04B0902F
:105CA0004B04C0904C04D0904D04609168047091F6
:105CB000690480916A0490916B040E9499603B0191
:105CC0004C010027F7FC0095102FC801B7010E9476
:105CD0009960A60195010E94FD5F9B01AC01C40182
:105CE000B3010E94FE5F0E94666060936804709337
:105CF000690480936A0490936B048FEC80937A001C
:105D0000109227038091780490917904A0917A04ED
:105D1000B0917B048B8B9C8BAD8BBE8B8091700480
:105D200090917104A0917204B09173048F87988B45
:105D3000A98BBA8BA8A1B9A11D01442437FC4094BA
:105D4000542C8091800490918104A0918204B091A0
:105D50008304820D931DA41DB51D8B8F9C8FAD8F69
:105D6000BE8F8B879C87AD87BE878093800490937E
:105D70008104A0938204B093830460902209709000
:105D800023098090240990902509620C731C841CBF
:105D9000951C6F82788689869A8660922209709215
:105DA000230980922409909225099091B1049E8341
:105DB000992329F48091B204882309F4A0C4A09106
:105DC0006808A98310925F0810925E0810925B0821
:105DD00010925A0810921B0510921C0510921D0576
:105DE00010921E0510921F05109220051092210599
:105DF00010922205B091B903BF8FA0901B05B090FF
:105E00001C05C0901D05D0901E05E0901F05F09068
:105E100020050091210510912205C601B5012CE94C
:105E20003FEF4FEF5FEF0E94C16129014E0C5F1CF5
:105E30005092CD084092CC08C801B70124E630E06A
:105E400040E050E00E94C16119012A183B083092DD
:105E5000C2082092C108E090BD03F090BE030091FB
:105E6000BF031091C003C801B70128E631E040E04C
:105E700050E00E944D615B016C0166167706880652
:105E80009906B4F0C801B70128E93EEF4FEF5FEF84
:105E90000E944D61660D771D881D991D6093220932
:105EA0007093230980932409909325093B014C01A9
:105EB00097FC04C62F89388D240D351D79010027E4
:105EC000F7FC0095102F80917C0490917D04A091A7
:105ED0007E04B0917F048E0D9F1DA01FB11F809383
:105EE0007C0490937D04A0937E04B0937F04809102
:105EF000AD049091AE04281B390B442737FD409523
:105F0000542F8B899C89AD89BE89280F391F4A1F60
:105F10005B1F209378043093790440937A04509364
:105F20007B04E090A503F090A6030091A7031091D5
:105F3000A803E216F30604071507C4F488EA91E6FD
:105F4000A0E0B0E08E199F09A00BB10B80937804FC
:105F500090937904A0937A04B0937B0480937C049B
:105F600090937D04A0937E04B0937F0488279927A3
:105F7000DC018E199F09A00BB10B60907804709022
:105F8000790480907A0490907B04681679068A06DA
:105F90009B06C4F4D801C701885A9146A040B0407E
:105FA0008093780490937904A0937A04B0937B044F
:105FB00080937C0490937D04A0937E04B0937F042F
:105FC0003C014D01298D3A8D220D331D79010027A9
:105FD000F7FC0095102F8091740490917504A091A6
:105FE0007604B09177048E0D9F1DA01FB11F809382
:105FF000740490937504A0937604B0937704809111
:10600000AF049091B004281B390B442737FD40950D
:10601000542F8F859889A989BA89280F391F4A1F5B
:106020005B1F20937004309371044093720450936B
:106030007304E090A103F090A2030091A3031091D8
:10604000A403E216F30604071507C4F488EA91E6F0
:10605000A0E0B0E08E199F09A00BB10B80937004F3
:1060600090937104A0937204B093730480937404AA
:1060700090937504A0937604B093770488279927AA
:10608000DC018E199F09A00BB10B20917004309197
:1060900071044091720450917304281739074A071C
:1060A0005B07C4F4D801C701885A9146A040B040AC
:1060B0008093700490937104A0937204B09373045E
:1060C0008093740490937504A0937604B09377043E
:1060D0009C01AD018B8D9C8DAD8DBE8D80936C042C
:1060E00090936D04A0936E04B0936F0420935004BA
:1060F00030935104409352045093530460925804D7
:106100007092590480925A0490925B0480917404B6
:1061100090917504A0917604B09177048093540413
:1061200090935504A0935604B093570480917C0437
:1061300090917D04A0917E04B0917F0480935C04D3
:1061400090935D04A0935E04B0935F0480911A0362
:1061500090911B0397FDCCC4959587959595879550
:10616000959587959093CF088093CE0880911C03D6
:1061700090911D0397FDBAC4959587959595879540
:10618000959587959093C0088093BF0880910704E8
:10619000909108040F9734F488E19CEF9093CF0816
:1061A0008093CE088091070490910804079734F4F7
:1061B00080E398EF9093CF088093CE082091080158
:1061C0002A3009F4F9C18091070490910804815D97
:1061D000974034F088EE93E09093CF088093CE08F8
:1061E0008091070490910804805E97400CF0F9C1FB
:1061F0008091090490910A040F9734F488E19CEF90
:106200009093C0088093BF088091090490910A047C
:10621000079734F480E398EF9093C0088093BF0809
:106220002A3009F4ADC18091090490910A04815D7E
:10623000974034F088EE93E09093C0088093BF08B5
:106240008091090490910A04805E97400CF0ADC1E2
:106250006091B003662309F4A2C040911A035091E3
:106260001B038091110590911205481B590B509307
:106270000C0540930B0520911A0330911B03280F46
:10628000391F37FD3FC4359527953093120520936C
:106290001105413851050CF427C280E890E0909335
:1062A0000C0580930B05E62FF0E080910B05909193
:1062B0000C05E89FB001E99F700DF89F700D112447
:1062C0009B0177FD2AC435952795359527953595FA
:1062D0002795359527958091CE089091CF08820F0C
:1062E000931F9093CF088093CE0840911C03509148
:1062F0001D0380910F0590911005481B590B509379
:106300000E0540930D0520911C0330911D03280FAD
:10631000391F37FD08C43595279530931005209314
:106320000F05413851050CF4D6C380E890E09093F6
:106330000E0580930D0580910D0590910E05E89F47
:10634000A001E99F500DF89F500D11249A0157FDAF
:10635000E7C3359527953595279535952795359537
:1063600027958091BF089091C008820F931F90934A
:10637000C0088093BF0880911A0390911B03680F97
:10638000791F70931B0360931A0380911C039091F3
:106390001D03480F591F50931D0340931C038F8901
:1063A000988D181619060CF0FFC220915A083091EA
:1063B0005B0837FDAEC3B901882777FD8095982F1C
:1063C000AF8D2A2F30E040E050E00E944D6120E484
:1063D00030E040E050E00E94C161420E531E5092F6
:1063E000CD084092CC08E98DFA8D1E161F060CF0E0
:1063F00006C320915E0830915F0837FD86C3B9015E
:10640000882777FD8095982FFF8D2F2F30E040E073
:1064100050E00E944D6120E430E040E050E00E94F6
:10642000C161220E331E3092C2082092C108B98188
:10643000B7FD0DC380916408E82FF0E0EE0FFF1F59
:10644000E25DF74F80819181A0919704B09198040B
:1064500083599F4F8A179B070CF41EC1CD010196EB
:106460009093980480939704DC0180916508E82F4D
:10647000F0E0EE0FFF1FE25DF74F808191816091A8
:10648000990470919A0483599F4F861797070CF4CB
:10649000EFC0CB01019690939A0480939904BC01BC
:1064A00080916608E82FF0E0EE0FFF1FE25DF74FE6
:1064B0008081918140919B0450919C0483599F4F0E
:1064C000841795070CF4C0C0CA01019690939C04F0
:1064D00080939B04AC0180916708E82FF0E0EE0FF9
:1064E000FF1FE25DF74F8081918120919D043091E3
:1064F0009E0483599F4F821793070CF479C0C901FA
:10650000019690939E0480939D049C01B7FD85C0E5
:10651000AF3FB10511F00CF0E0C077FD84C06F3FD4
:10652000710511F00CF0D2C057FD83C04F3F5105EB
:1065300011F00CF0C4C037FD82C02F3F310539F097
:1065400034F08FEF90E090939E0480939D04A19689
:106550000FB6F894DEBF0FBECDBFCF91DF911F9174
:106560000F91FF90EF90DF90CF90BF90AF909F90F2
:106570008F907F906F905F904F903F902F900895F5
:106580008091090490910A04835F934034F088EE6F
:1065900093E09093C0088093BF0880910904909184
:1065A0000A048A5F93400CF453CE80ED97E09093F9
:1065B000C0088093BF084CCE8091070490910804D6
:1065C000835F934034F088EE93E09093CF088093FC
:1065D000CE0880910704909108048A5F93400CF4E0
:1065E00007CE80ED97E09093CF088093CE0800CE41
:1065F0008081918182599F4F821793070CF086CF3B
:106600002115310509F482CFC901019790939E04A9
:1066100080939D049C01B7FF7BCF10929804109249
:10662000970477FF7CCF10929A041092990457FF39
:106630007DCF10929C0410929B0437FF7ECF109266
:106640009E0410929D0483CF8081918182599F4F37
:10665000841795070CF03FCF4115510509F43BCF46
:10666000CA01019790939C0480939B04AC0133CFA3
:106670008081918182599F4F861797070CF010CF28
:106680006115710509F40CCFCB01019790939A0421
:1066900080939904BC0104CF8081918182599F4FDE
:1066A0008A179B070CF0E1CE109709F4DECECD01DE
:1066B00001979093980480939704DC01D6CE8FEFD6
:1066C00090E090939C0480939B0435CF8FEF90E0F3
:1066D00090939A048093990427CF8FEF90E0909342
:1066E00098048093970419CF40585F4F0CF0DBCD8E
:1066F00080E89FEF90930C0580930B05D4CDB0916B
:106700006808B983B6FF5ECB2B893C894D895E89C9
:10671000283BE4E93E07EEEF4E07EFEF5E0724F477
:1067200028EB34E94EEF5FEF2A833B834C835D8394
:1067300029543B464140504044F088E49BE6A1E0A8
:10674000B0E08A839B83AC83BD832F8538894989D8
:106750005A89283B94E939079EEF49079FEF59076B
:1067600024F428EB34E94EEF5FEF39014A01293474
:10677000ABE63A07A1E04A07A0E05A073CF038E44C
:10678000632E3BE6732E31E0832E912CA090B8034C
:10679000BB24CC24DD24EF89F88D9F01442737FDED
:1067A0004095542FC401B3010E944D6120E038E0B0
:1067B00040E050E00E94C161CA01B901A601950103
:1067C0000E944D6120E030E140E050E00E94C16154
:1067D00079018A01E0921705F092180500931905D6
:1067E00010931A05898D9A8D9C01442737FD409599
:1067F000542F6A817B818C819D810E944D6120E0B4
:1068000038E040E050E00E94C161CA01B901A60130
:1068100095010E944D6120E030E140E050E00E948F
:10682000C161C901DA01F0925B08E0925A08309325
:106830005F0820935E085C016D01AE18BF08C00AB6
:10684000D10AA0921305B0921405C0921505D092FA
:1068500016058F819885A985BA858A0D9B1DAC1D6B
:10686000BD1D8093220990932309A0932409B0931E
:1068700025099091B9039F8F9923E1F4C601B501D1
:1068800022E030E040E050E00E94C1618B859C85B1
:10689000AD85BE85821B930BA40BB50B8093800442
:1068A00090938104A0938204B09383048B8F9C8F78
:1068B000AD8FBE8FA20CB31CC41CD51CE090B703D7
:1068C000FF2400E010E0C601B501A40193010E947D
:1068D0004D6120E038E040E050E00E94C161CA0113
:1068E000B901A80197010E944D6120E030E140E02C
:1068F00050E00E94C161922E832E742E652E20934B
:106900001F05309320054093210550932205C601B1
:10691000B5012A813B814C815D810E944D6120E05F
:1069200038E040E050E00E94C161CA01B901A8010D
:1069300097010E944D6120E030E140E050E00E946C
:10694000C161B901FA0120931B0570931C054093A6
:106950001D05F0931E0588A199A197FD19C18134E9
:106960009105CCF0292D382D472D562DC901DA017E
:10697000B7FDF1C081389105A105B1054CF4CB01FB
:10698000DF01B7FD09C181389105A105B1051CF0F2
:1069900081E0809394046090220970902309809094
:1069A00024099090250929CA20915A0830915B0842
:1069B00037FDC0C0B901882777FD8095982FBF8D1E
:1069C0002B2F30E040E050E00E944D6120E430E0A9
:1069D00040E050E00E94C16150954095309521956E
:1069E0003F4F4F4F5F4F420E531E5092CD08409283
:1069F000CC08E98DFA8D1E161F060CF4FACC2091F6
:106A00005E0830915F0837FD91C0B901882777FD96
:106A10008095982FAF8D2A2F30E040E050E00E9403
:106A20004D6120E430E040E050E00E94C1615095AB
:106A30004095309521953F4F4F4F5F4F220E331EAB
:106A40003092C2082092C108B981B7FFF3CCEE8121
:106A5000EE2309F0EFCC8091B204882309F0EACC50
:106A6000298D3A8D61E0213036070CF067C0898DA1
:106A70009A8D80509F4F74F48091CE089091CF08EA
:106A800080509F4FE98DFA8D8E0F9F1F9093CF08F6
:106A90008093CE082F89388D61E0213036070CF4C1
:106AA00062C08091BF089091C00880509140820FD1
:106AB000931F9093C0088093BF08BCCC6A0C7B1CCA
:106AC0008C1C9D1C609222097092230980922409DB
:106AD00090922509EFC940585F4F0CF02CCC80E80C
:106AE0009FEF90930E0580930D0525CC079644CB20
:106AF000079632CB295F3F4F0C94432D295F3F4FC0
:106B00000C94322D2F5F3F4FBECB309521953F4FD8
:106B100076CC309521953F4F4ECC215F3F4FD3CB64
:106B2000215F3F4F16CC2F5F3F4FF5CB309521951E
:106B30003F4F6BCF309521953F4F3CCF8091CE0892
:106B40009091CF0880509140820F931F9093CF086F
:106B50008093CE089FCFB095A095909581959F4F3B
:106B6000AF4FBF4F07CF8F89988D80509F4F0CF04C
:106B700061CC8091BF089091C00880509F4FEF89F1
:106B8000F88D8E0F9F1F9093C0088093BF0852CC42
:106B9000909581959F4FE3CEB095A0959095819566
:106BA0009F4FAF4FBF4FEFCE80916B088B3F80F070
:106BB0008B3F09F4A3C28C3F09F4EAC38D3F09F46B
:106BC0002EC38E3F39F480919D048093AC0302C0A4
:106BD0008093AC0380916A088B3F80F08B3F09F46F
:106BE0007EC28C3F09F4D9C38D3F09F413C38E3F95
:106BF00039F480919D048093AB0302C08093AB0372
:106C00008091AB038823B1F41092AB0380916C08A0
:106C10008B3FC8F08B3F09F467C28C3F09F4C2C3B5
:106C20008D3F09F406C38E3F81F480919D048093CB
:106C3000AD030BC0843650F384E68093AB038091A0
:106C40006C088B3F38F78093AD038091AD038823A8
:106C5000B1F41092AD0380916E088B3FC8F08B3F6A
:106C600009F447C28C3F09F4B1C38D3F09F4DCC27B
:106C70008E3F81F480919D048093AE030BC08436D7
:106C800050F384E68093AD0380916E088B3F38F714
:106C90008093AE03809175088B3F80F08B3F09F4A1
:106CA0008CC28C3F09F48DC38D3F09F4D1C28E3F55
:106CB00039F480919D048093AF0302C08093AF03A9
:106CC000809176088B3F80F08B3F09F47BC28C3F2C
:106CD00009F42CC38D3F09F4C0C28E3F39F4809172
:106CE0009D048093B10302C08093B1038091B103EE
:106CF0008B30B8F48AE08093B103809177088B3FA2
:106D0000C0F08B3F09F463C28C3F09F414C38D3F7C
:106D100009F4CBC28E3F79F480919D048093B20335
:106D20000AC08F3F51F78093B103809177088B3F62
:106D300040F78093B203809178088B3F80F08B3FBF
:106D400009F422C28C3F09F400C38D3F09F4A8C2A4
:106D50008E3F39F480919D048093B00302C08093EC
:106D6000B00380917D088B3F80F08B3F09F411C206
:106D70008C3F09F4BDC28D3F09F4A6C28E3F39F4A1
:106D800080919D048093B40302C08093B4038091EA
:106D90007E088B3F80F08B3F09F400C28C3F09F4E2
:106DA000CFC28D3F09F495C28E3F39F480919D0486
:106DB0008093B70402C08093B70480917F088B3F13
:106DC00080F08B3F09F4CCC18C3F09F48CC28D3F1D
:106DD00009F475C28E3F39F480919D048093B80404
:106DE00002C08093B804809180088B3F80F08B3F75
:106DF00009F4BBC18C3F09F494C28D3F09F45AC217
:106E00008E3F39F480919D048093B90402C0809331
:106E1000B904809181088B3F80F08B3F09F4AAC1AF
:106E20008C3F09F479C28D3F09F430C28E3F39F4AA
:106E300080919D048093BA0402C08093BA0480912B
:106E400092088B3F80F08B3F09F499C18C3F09F485
:106E500090C28D3F09F41FC28E3F39F480919D048A
:106E60008093BB0402C08093BB04809193088B3F46
:106E700080F08B3F09F44CC18C3F09F47FC28D3FF9
:106E800009F4C3C18E3F39F480919D048093BC0402
:106E900002C08093BC04809194088B3F80F08B3FAC
:106EA00009F43BC18C3F09F432C28D3F09F4A8C1FB
:106EB0008E3F39F480919D048093BD0402C080937D
:106EC000BD04809195088B3F80F08B3F09F42AC167
:106ED0008C3F09F417C28D3F09F4CEC18E3F39F4BF
:106EE00080919D048093BE0402C08093BE04809173
:106EF00082088B3F80F08B3F09F419C18C3F09F465
:106F00006AC28D3F09F4BDC18E3F39F480919D0462
:106F10008093B50302C08093B503809187088B3FAF
:106F200080F08B3F09F408C18C3F09F4E6C18D3F26
:106F300009F49DC18E3F39F480919D048093B6037E
:106F400002C08093B60380918A088B3F80F08B3F0C
:106F500009F4F7C08C3F09F407C28D3F09F482C1E0
:106F60008E3F39F480919D048093B70302C08093D3
:106F7000B70380918B088B3F80F08B3F09F4E6C00C
:106F80008C3F09F4ECC18D3F09F430C18E3F39F4D8
:106F900080919D048093B80302C08093B8038091D0
:106FA0008C088B3F80F08B3F09F4D5C08C3F09F4EF
:106FB000FEC18D3F09F41FC18E3F39F480919D04BD
:106FC0008093B90302C08093B903809191088B3FED
:106FD00080F08B3F09F4E7C08C3F09F4EDC18D3F91
:106FE00009F431C18E3F39F480919D048093BA0336
:106FF00002C08093BA03809197088B3F80F08B3F4B
:1070000009F4D6C08C3F09F4BEC18D3F09F416C106
:107010008E3F39F480919D048093E60802C08093EE
:10702000E6088091E608823008F455C08F3F09F4E5
:107030004BC0809199088B3F80F08B3F09F463C06F
:107040008C3F09F487C18D3F09F4CBC08E3F39F4E2
:1070500080919D048093190902C080931909809141
:1070600019098230A0F18F3F61F18091AA088B3F0E
:1070700080F08B3F09F4B0C08C3F09F4B1C18D3F63
:1070800009F42CC18E3F39F480919D048093290925
:1070900002C0809329096091B40370E06F5F7F4F55
:1070A0008CE398E20E948C617093AA036093A90319
:1070B0008091730880931A09809172088093D30895
:1070C000089580931909D1CF8093E608B2CF81E06B
:1070D00080931909CACF81E08093E608AACF8091F6
:1070E00097048093AB038CCD809197048093AD037C
:1070F000ACCD809197048093AE03CCCD8091970462
:107100008093AC0367CD8091970480931909A7CF32
:10711000809197048093BC04BECE809197048093A5
:10712000BD04CFCE809197048093BE04E0CE8091C1
:1071300097048093B503F1CE809197048093B603B2
:1071400002CF809197048093B70313CF8091970467
:107150008093B80324CF809197048093B90335CFEF
:10716000809197048093B8043ECE809197048093D9
:10717000B9044FCE809197048093BA0460CE809179
:1071800097048093BB0471CE809197048093B003E1
:10719000E8CD809197048093B403F9CD8091970452
:1071A0008093B7040ACE809197048093BA0323CFCB
:1071B000809197048093E60834CF80919704809360
:1071C000AF037ECD809197048093B1038FCD8091E2
:1071D00097048093B203AFCD8091970480932909DF
:1071E0005ACF80919B048093190939CF80919B04D9
:1071F0008093B803D4CE80919B048093B903E5CEED
:1072000080919B048093BD045CCE80919B0480930D
:10721000BC0441CE80919B048093AB03F1CC809160
:107220009B048093AC03D6CC80919B048093AE03E7
:1072300031CD80919B048093AD0307CD80919B0459
:107240008093E608EECE80919B048093BA03D3CE60
:1072500080919B048093AF0333CD80919B048093F6
:10726000B10344CD80919B048093B70382CE80917B
:107270009B048093B60367CE80919B048093BE04E9
:1072800036CE80919B048093B50347CE80919B04BA
:107290008093BA04D4CD80919B048093BB04E5CD48
:1072A00080919B048093B0035CCD80919B0480937C
:1072B000B20341CD80919B048093B904AACD809103
:1072C0009B048093B8048FCD80919B048093B4037A
:1072D0005ECD80919B048093B7046FCD80919B0419
:1072E00080932909D8CE809199048093B8047BCDEE
:1072F000809199048093B4034ACD8091990480933E
:10730000B60321CE809199048093BE04F0CD809184
:1073100099048093BD04D5CD809199048093BA04DB
:107320008ECD809199048093B90473CD8091990496
:107330008093B103DBCC809199048093B203FBCCA2
:10734000809199048093B70438CD809199048093FB
:10735000B00307CD809199048093190980CE809164
:1073600099048093B8031BCE809199048093B7034E
:1073700000CE809199048093BB0477CD80919904CD
:107380008093BC0488CD809199048093E60849CE0F
:10739000809199048093AC031DCC809199048093D3
:1073A000AB032ECC809199048093AD034ECC809199
:1073B00099048093B90309CE809199048093BA030C
:1073C0001ACE809199048093AF037ACC809199046E
:1073D0008093AE035FCC809199048093B5039DCDDB
:1073E000809199048093290956CE8091A80488231E
:1073F000F1F48091CB048C7F8093CB0420E030E0CB
:107400000DC0D901AB51B94FF901E35FF64F8C9133
:1074100080832F5F3F4F2C30310561F18091DE0377
:10742000882379F7D901AB51B94F1C92EDCF8091E8
:10743000CB0481608093CB04EAEBF7E080910D09E7
:107440008093BA071092BB0780910E098093BC0706
:107450001382809110098093BE07158280910F09D5
:107460008093C007178210923104109232040E9458
:10747000122A08958091DE038823F1F28091DE03C1
:1074800081508093DE03D8CF809108018D3009F4BC
:1074900071C110927A008091070490910804909332
:1074A000CF088093CE088091090490910A049093AC
:1074B000C0088093BF0880910B0490910C049093B6
:1074C0001C0980931B0960910F0470911004882798
:1074D00077FD8095982F26E030E040E050E00E9454
:1074E0004D6170930B0960930A0960910D047091CE
:1074F0000E04882777FD8095982F0E944D61709328
:1075000027096093260980911104909112049093A9
:10751000DA088093D9088FEC80937A008091640810
:10752000E82FF0E0EE0FFF1FE25DF74F80819181C1
:10753000A0919704B091980483599F4F8A179B0795
:107540000CF4F0C0CD0101969093980480939704B9
:10755000DC0180916508E82FF0E0EE0FFF1FE25D8F
:10756000F74F808191816091990470919A048359B9
:107570009F4F861797070CF4C1C0CB0101969093DB
:107580009A0480939904BC0180916608E82FF0E08A
:10759000EE0FFF1FE25DF74F8081918140919B04C8
:1075A00050919C0483599F4F841795070CF492C007
:1075B000CA01019690939C0480939B04AC01809136
:1075C0006708E82FF0E0EE0FFF1FE25DF74F8081C4
:1075D000918120919D0430919E0483599F4F821781
:1075E00093070CF44BC0C901019690939E048093BD
:1075F0009D049C01B7FD57C0AF3FB10511F00CF0E1
:10760000B2C077FD56C06F3F710511F00CF0A4C0F9
:1076100057FD55C04F3F510511F00CF096C037FD96
:1076200054C02F3F310539F034F08FEF90E0909344
:107630009E0480939D0460918D0870E080E090E04E
:1076400024EC39E040E050E00E944D616093A103DA
:107650007093A2038093A3039093A40360918E0878
:1076600070E080E090E00E944D616093A50370930C
:10767000A6038093A7039093A80308958081918126
:1076800082599F4F821793070CF0B4CF2115310513
:1076900009F4B0CFC901019790939E0480939D0493
:1076A0009C01B7FFA9CF109298041092970477FF1E
:1076B000AACF10929A041092990457FFABCF109260
:1076C0009C0410929B0437FFACCF10929E04109242
:1076D0009D04B1CF8081918182599F4F8417950776
:1076E0000CF06DCF4115510509F469CFCA0101971E
:1076F00090939C0480939B04AC0161CF8081918125
:1077000082599F4F861797070CF03ECF6115710580
:1077100009F43ACFCB01019790939A04809399048E
:10772000BC0132CF8081918182599F4F8A179B077C
:107730000CF00FCF109709F40CCFCD010197909367
:10774000980480939704DC0104CF8FEF90E090932E
:107750009C0480939B0463CF8FEF90E090939A04F6
:107760008093990455CF8FEF90E090939804809385
:10777000970447CF0E94841F8CCE6F927F928F9286
:107780009F92AF92BF92CF92DF92EF92FF920F93B0
:107790001F93CF93DF931092F103469A1092450402
:1077A00010924404109247041092460480E090E046
:1077B000A0E0B0E080934A0490934B04A0934C0463
:1077C000B0934D0410923B0410923A0410923D0481
:1077D00010923C0410923F0410923E041092EC0868
:1077E0001092EB081092B7031092B8031092140491
:1077F0000E94443A84E690E00E9420170E94443A96
:107800008091680880FF10C080912203909123032B
:10781000875B934008F0FFC180912203909123037E
:107820008E5E924008F4F7C1AA24EE24FF24C0E043
:10783000D0E000E010E08AE090E00E942017809104
:107840000B0490910C04E80EF91E809107049091AE
:107850000804C80FD91F8091090490910A04080FE9
:10786000191FA39480E2A81631F7AE01405F5F4F65
:10787000569547955695479550933B0440933A0447
:107880009801205F3F4F3695279536952795309381
:107890003D0420933C04C7014096969587959295A8
:1078A00082958F7089279F70892790933F048093DA
:1078B0003E049093EC088093EB08309341042093AE
:1078C00040045093430440934204F999FECF24E0CE
:1078D00030E032BD21BDF89A80B5853008F09EC1F8
:1078E000F999FECF32BD21BDF89A30B5F999FECF96
:1078F00085E090E092BD81BDF89A20B5932F80E09D
:10790000820F911D9093450480934404F999FECF12
:1079100086E090E092BD81BDF89A30B5F999FECF2E
:1079200087E090E092BD81BDF89A20B5932F80E06A
:10793000820F911D9093470480934604F999FECFDE
:1079400088E090E092BD81BDF89A30B5F999FECFFC
:1079500089E090E092BD81BDF89A20B5732F60E078
:10796000620F711D882777FD8095982F0E9499607E
:1079700060934A0470934B0480934C0490934D049D
:107980001092CF081092CE081092C0081092BF0833
:1079900010921C0910921B0984E690E00E942017A7
:1079A00060910F0470911004882777FD8095982FBF
:1079B00026E030E040E050E00E944D613B014C0188
:1079C00070930B0960930A0960910D0470910E0485
:1079D000882777FD8095982F0E944D615B016C018F
:1079E0007093270960932609E0907408FF2400E053
:1079F00010E0882477FC8094982CC401B301A8017E
:107A000097010E944D613B014C01609350047093BB
:107A100051048093520490935304CC24B7FCC09437
:107A2000DC2CC601B5010E944D616093580470932F
:107A3000590480935A0490935B046092740470928A
:107A40007504809276049092770460937C0470931E
:107A50007D0480937E0490937F04109280041092A2
:107A60008104109282041092830480911E039091ED
:107A70001F03A0912003B09121039093E907809305
:107A8000E8071092160410921504109288041092C0
:107A9000890410928A0410928B0480918C04909136
:107AA0008D0490938F0480938E040E942B5982E35F
:107AB00090E09093EF038093EE0360918D0870E067
:107AC00080E090E024EC39E040E050E00E944D611D
:107AD0006856754C8F4F9F4F6093A1037093A2031C
:107AE0008093A3039093A40360918E0870E080E0DC
:107AF00090E00E944D616856754C8F4F9F4F609388
:107B0000A5037093A6038093A7039093A8031092F4
:107B1000BC031092BB0360918C0470918D04882784
:107B200077FD8095982F2091BD033091BE03409141
:107B3000BF035091C0030E944D616093220970936E
:107B4000230980932409909325091092960410929A
:107B5000950411E0109309010E94995C8091CB0477
:107B600084608093CB048FEF80938B0910928C09F3
:107B700080E280938D09E0916408F0E0EE0FFF1F32
:107B8000E25DF74F8081918182599F4F90939804D5
:107B900080939704E0916508F0E0EE0FFF1FE25D2F
:107BA000F74F8081918182599F4F90939A048093DF
:107BB0009904E0916608F0E0EE0FFF1FE25DF74FD9
:107BC0008081918182599F4F90939C0480939B0464
:107BD000E0916708F0E0EE0FFF1FE25DF74F808154
:107BE000918182599F4F90939E0480939D0410939E
:107BF000F10384E680939F04DF91CF911F910F9151
:107C0000FF90EF90DF90CF90BF90AF909F908F90BC
:107C10007F906F9008950E94752006CE809126096E
:107C20009091270997FD29C06CE070E00E948C615B
:107C3000709347046093460480910A0990910B0960
:107C400097FD1FC06CE070E00E948C61709345044A
:107C5000609344046091E6077091E707882777FDF9
:107C60008095982F0E94996060934A0470934B040A
:107C700080934C0490934D0483CE909581959F4FB3
:107C8000D3CF909581959F4FDDCF1F93CF93DF93F7
:107C9000982F8823C1F08091A8048823A1F4192F7C
:107CA0001150C4E6D0E005C011508091A80488238B
:107CB00051F4D093EF03C093EE038AEF90E00E945B
:107CC0000A17112389F7DF91CF911F9108952F9201
:107CD0003F924F925F926F927F928F929F92AF925C
:107CE000BF92CF92DF92EF92FF920F931F93DF9399
:107CF000CF93CDB7DEB7C154D0400FB6F894DEBFF6
:107D00000FBECDBF0E94002D409108014C3010F0F5
:107D10000C949749299A2091A6043091A7043E8398
:107D20002D838091D308282F30E0C90109966D81F9
:107D30007E818617970724F0C9010A969E838D835A
:107D400080919F04843610F00C94CE4780910D01F1
:107D5000882349F480911103909112038F5F9F4F04
:107D600011F40C94A7518091ED049091EE040097CA
:107D700011F00C9498501092A804109292044A307A
:107D800011F40C94A150443111F40C94A150289892
:107D90008091C9049091CA04895E934010F40C94B8
:107DA000B45080917A08E82FF0E0FE83ED8381E003
:107DB00080939204A0916008B0E0AA0FBB1FFD0160
:107DC000EC5BF74F11821082E09161082E2F30E0BA
:107DD000220F331FC9018C5B974FFC011182108267
:107DE000A25DB74F11961C921E92225D374FD901AA
:107DF00011961C921E92E0916308F0E0EE0FFF1FB7
:107E0000E25DF74F1182108280918303815080934D
:107E100083038F5F31F0509192045EA7552309F4DC
:107E20002BC20E94D435E0916008F0E0EE0FFF1FF6
:107E3000E25DF74F2081318180916F0890E0289FAB
:107E4000A001299F500D389F500D11242091DC0472
:107E50003091DD04C901880F991F820F931F480FCD
:107E6000591F57FF02C00C94FB51559547955595E6
:107E700047955093DD044093DC04E0916008F0E006
:107E8000EE0FFF1FEC5BF74F20813181809170086E
:107E900090E0BC01269FC001279F900D369F900D5A
:107EA0001124840F951F9093DD048093DC042091AE
:107EB0002705309128054091230550912405821B08
:107EC000930B841B950B9093A1048093A004E091E5
:107ED0006108F0E0EE0FFF1FE25DF74F2081318176
:107EE00080916F0890E0289FA001299F500D389F36
:107EF000500D11242091DA043091DB04C901880F60
:107F0000991F820F931F480F591F57FF02C00C94EF
:107F1000FF5155954795559547955093DB044093F0
:107F2000DA04E0916108F0E0EE0FFF1FEC5BF74F21
:107F3000208131818091700890E0DC012A9FC0018E
:107F40002B9F900D3A9F900D1124840F951F9093B5
:107F5000DB048093DA042091290530912A054091B1
:107F6000250550912605821B930B841B950B90933E
:107F7000A3048093A204E0916308F0E0EE0FFF1FDA
:107F8000E25DF74F8081918122273327281B390B2F
:107F90002330310514F40C94F64A225030403093CB
:107FA000A5042093A404E0916208F0E0EE0FFF1F07
:107FB000E25DF74F0081118108581F4F1093A7040D
:107FC0000093A6046091B10370E0882777FD809547
:107FD000982F0E94996020E030E040E251E40E9436
:107FE000FE5F0E946B60609320092091B203209392
:107FF000ED086093C6082093DD088091070780FF95
:1080000006C080912909813810F00C94C8508091E5
:10801000A6049091A70497FF02C00C94E3518091AD
:10802000680882FF02C01092ED086091A004709170
:10803000A1044091C5045091C604CB019C0197FF57
:1080400002C00C94F751359527953595279537FF44
:1080500002C00C94F2514217530714F00C94AC5028
:108060009B0177FF02C00C941B52C901959587951F
:10807000959587959093C6048093C50485369105A0
:1080800014F00C945C516091A2047091A30440918F
:10809000C7045091C804CB019C0197FF02C00C9407
:1080A000EE51359527953595279537FF02C00C94ED
:1080B000E9514217530714F00C94A4509B0177FF29
:1080C00002C00C941652C901959587959595879590
:1080D0009093C8048093C7048536910514F00C94DE
:1080E0005451509192045EA7552341F01092C6045A
:1080F0001092C5041092C8041092C70480916108C0
:10810000A82FB0E0AA0FBB1FFD01E25DF74F208151
:10811000318180918808482F50E04217530734F48A
:108120008091AB0882FF02C00C944F51FD01E25DCB
:10813000F74F2081318180918908BA01681B71094C
:108140002617370764F41092B30480916108A82FB2
:10815000B0E080918808482F50E0AA0FBB1FFD01B6
:10816000E25DF74F2081318188279927841B950B89
:108170002817390734F48091AB0883FF02C00C94B0
:1081800046518091B404882371F0A25DB74F2D91C0
:108190003C918091890890E0841B950B821793078E
:1081A00014F40C948D5180916008A82FB0E0AA0FB0
:1081B000BB1FFD01E25DF74F808191814817590790
:1081C00034F48091AB0880FF02C00C943C51609164
:1081D000B604662379F0FD01E25DF74F208131811D
:1081E00080918908FA01E81BF1092E173F0714F462
:1081F0000C947E51FD01E25DF74F2081318188278B
:108200009927841B950B2817390734F48091AB0804
:1082100081FF02C00C9437518091B504882371F01E
:10822000A25DB74F2D913C918091890890E0841B0D
:10823000950B8217930714F40C9495518091B30415
:10824000882331F48091B404882311F40C943351C1
:1082500081E08093B204662331F48091B5048823D1
:1082600011F40C942F5181E08093B1041092B20468
:108270001092B3041092B404F091B204FB8BFF236C
:1082800009F0EBC78091B104882309F0E6C73EA549
:108290003323D9F01092A5041092A4041092A104E3
:1082A0001092A0041092A3041092A2049AE5909355
:1082B000200988E78093ED089093C6088093DD0835
:1082C0001092B2041092B1041B8A4091E0085091C0
:1082D000E1086091E2087091E3084D8F5E8F6F8F27
:1082E00078A3609150047091510480915204909150
:1082F00053046D8B7E8B8F8B988F2D8D3E8D4F8D84
:1083000058A1260F371F481F591F2093E0083093AC
:10831000E1084093E2085093E3082090E70830908A
:10832000E8084090E9085090EA08409158045091BC
:10833000590460915A0470915B0448AB59AB6AAB25
:108340007BAB240E351E461E571E2092E708309246
:10835000E8084092E9085092EA088091D508909187
:10836000D608A091D708B091D80820915404309134
:1083700055044091560450915704298F3A8F4B8FE2
:108380005C8F820F931FA41FB51F8093D508909315
:10839000D608A093D708B093D8088091C7089091C9
:1083A000C808A091C908B091CA0840915C045091D6
:1083B0005D0460915E0470915F044AA35BA36CA3AB
:1083C0007DA3840F951FA61FB71F8093C7089093A6
:1083D000C808A093C908B093CA085091B1045EA31D
:1083E000552329F46B89662311F40C948E4F109257
:1083F000600410926104109262041092630410925F
:10840000640410926504109266041092670410923E
:10841000E0081092E1081092E2081092E30810922E
:10842000E7081092E8081092E9081092EA08109202
:10843000D5081092D6081092D7081092D80810923A
:10844000C7081092C8081092C9081092CA088091F3
:10845000700490917104A0917204B09173048093A0
:10846000740490937504A0937604B093770480917C
:10847000780490917904A0917A04B0917B04809360
:108480007C0490937D04A0937E04B0937F041092AB
:108490001804109217041092B0041092AF041092B6
:1084A000AE041092AD047EA1772311F40C94894F91
:1084B00080911704909118048F3F910511F008F0F6
:1084C00039C7309194043C8B4091ED084FA3E09064
:1084D000A404F090A504C701F7FCB3C7409764F06B
:1084E00088EE93E09093A00380939F0380916808A7
:1084F00084FD02C00C94324F10917108B701882797
:1085000077FD8095982F212F30E040E050E00E94C9
:108510004D61F701F7FE02C00C94BC509F01442747
:1085200037FD4095542F0E944D6120E032E040E03D
:1085300050E00E94C161812F90E08E9DB0018F9D1F
:10854000700D9E9D700D112477FF02C00C94B850E1
:108550007595679575956795260F371FC901AA27E9
:1085600097FDA095BA2F8093FF0490930005A093E8
:108570000105B0930205209180043091810440915F
:10858000820450918304281B390B4A0B5B0B209308
:1085900080043093810440938204509383042135F6
:1085A00063EC360760E0460760E056070CF4A9C7A5
:1085B00080E593ECA0E0B0E0809380049093810488
:1085C000A0938204B093830440908C0450908D0457
:1085D0004114510431F08091680883FF02C00C946B
:1085E000FA4D80901B0990901C098091E7048150FE
:1085F0008093E7048F5F09F0B1C088E18093E704BE
:10860000E0907408FF24EE0CFF1CEE0CFF1C00270A
:10861000F7FC0095102F6D897E898F89988DA801B0
:1086200097010E94C1613093A3072093A20768A914
:1086300079A98AA99BA9A80197010E94C1613093D9
:10864000A5072093A40720910A0930910B09C901BD
:1086500097FF02C00C94A0519595879595958795A5
:108660009093A7078093A6078091260990912709E8
:108670009C0137FF02C00C94A35135952795359581
:1086800027953093A9072093A8079092AB07809273
:10869000AA072091A9043091AA043093AD07209332
:1086A000AC078091E6079091E7079093AF0780931E
:1086B000AE075092B3074092B20780911803909191
:1086C00019039093B5078093B407609122097091C4
:1086D000230980912409909125092091BD033091AF
:1086E000BE034091BF035091C0030E94C16130930B
:1086F000B9072093B80780919F04E6EBF7E08093D9
:10870000B6071092B7078091FB068093C807138ABB
:108710008091F2039091F3039093CB078093CA0763
:1087200080918C09992787FD90959093D907809324
:10873000D80780918E098093DC0717A280912305CA
:10874000909124059093DF078093DE0780912505A3
:10875000909126059093E1078093E007FC89FF2321
:1087600081F01092030510920405109205051092F5
:10877000060510920705109208051092090510923F
:108780000A052EA1222309F497C61C821B826624A7
:1087900077244B89442309F47AC61A821982222449
:1087A00033242091C1083091C208293C31050CF4D2
:1087B00060C688EC90E09093C2088093C10828ECD2
:1087C00030E08091CC089091CD0822969FAF8EAF7B
:1087D0002297893C91050CF439C688EC90E090937F
:1087E000CD088093CC0822969FAF8EAF2297790157
:1087F0000027F7FC0095102FEE0CFF1C001F111F27
:10880000EE0CFF1C001F111FEE0CFF1C001F111FA0
:10881000EE0CFF1C001F111FEE0CFF1C001F111F90
:10882000EE0CFF1C001F111FEE0CFF1C001F111F80
:10883000A0902009BB24CC24DD244090CE08509089
:10884000CF089201442737FD4095542FC601B5014A
:108850000E944D61E60EF71E081F191FC801B701DF
:1088600020E430E040E050E00E94C1612301420E6C
:10887000531E5092CF084092CE0822962EAD3FADA7
:10888000229779010027F7FC0095102FEE0CFF1CB2
:10889000001F111FEE0CFF1C001F111FEE0CFF1C10
:1088A000001F111FEE0CFF1C001F111FEE0CFF1C00
:1088B000001F111FEE0CFF1C001F111FEE0CFF1CF0
:1088C000001F111F4091BF085091C008BA019B01C1
:1088D000442737FD4095542FC601B5010E944D61D4
:1088E000E60EF71E081F191FC801B70120E430E08B
:1088F00040E050E00E94C1616101C20ED31ED9A6C2
:10890000C8A6D092C008C092BF08880C991CB401B8
:10891000882777FD8095982F2091C60830E040E0A9
:1089200050E00E944D6120E430E040E050E00E94C1
:10893000C16179018A016091DD0870E080E090E01A
:1089400020916C0430916D0440916E0450916F043D
:108950000E944D6120EF35E540E050E00E94C1618A
:108960004701820E931E90921C0980921B0971E0B0
:10897000471670E457060CF422C680E090E490930A
:10898000CF088093CE08412CA0E45A2E91E0C9165E
:1089900090E4D9060CF404C680E090E49093C008FB
:1089A0008093BF0899A788A7B1E08B16B0E49B0617
:1089B0000CF497C580E090E490931C0980931B0908
:1089C000812CE0E49E2E80913404882349F080912C
:1089D000C9049091CA040297C09710F40C94754F83
:1089E0006D807E80660C771C660C771C8091680811
:1089F00080FFC7C081FF02C00C94374F8091AC0349
:108A00002091BB033091BC03280F311D80916D086C
:108A100090E0BC01269FC001279F900D369F900DCE
:108A2000112444979093AC048093AB0481E080932D
:108A300093042091A9043091AA047EA5772321F004
:108A40001092AC041092AB044091AB045091AC0472
:108A5000421753070CF095C080919304882309F4C2
:108A600090C08091AD0390E0241B350B829FA00144
:108A7000839F500D929F500D112457FF02C00C94FC
:108A8000D2545A01B594A794B594A794C0901504F4
:108A9000D0901604609188047091890480918A04B2
:108AA00090918B04E090AE03FF2400E010E020E8FA
:108AB00030E040E050E00E94C161C801B7010E946F
:108AC0004D6120E230E040E050E00E94C161B90118
:108AD0008EEF283E380714F468EE7EEF2091E8040C
:108AE0003091E904C901880F991F820F931FAC01CF
:108AF000440F551F440F551F480F591F9601D7FEAD
:108B000002C00C94CE5435952795421B530B4A193D
:108B10005B09CB01A1E069317A0714F088E191E0AB
:108B2000FA01E81BF90BCF01860D971D97FF02C0D4
:108B30000C94D654AC015595479555954795559548
:108B40004795559547955093E9044093E8048091E3
:108B50006908282F30E0220F331F220F331F4217DE
:108B6000530714F00C9424526216730614F00C94FC
:108B7000D5537092E9046092E8046090E804709024
:108B8000E904F0911A09FFA78F2F90E04497880F0E
:108B9000991F880F991F861597050CF43C01709258
:108BA000B1076092B0076091FF0470910005809159
:108BB0000105909102052CEF3FEF4FEF5FEF0E9410
:108BC0004D617401E60EF71E21EA621671040CF481
:108BD000A1C3B301759567956E157F050CF01AC595
:108BE0004FA5242F30E0220F331F220F331FC9015E
:108BF000861997097B01861797070CF47C01C3013E
:108C0000821B930B1701E816F9060CF41C018091E6
:108C1000A0049091A1049201281B390B3093DF0826
:108C20002093DE085FA1552309F45AC36B817C8130
:108C3000681B790BCB01AA2797FDA095BA2FE0906E
:108C40000705F09008050091090510910A05E80E46
:108C5000F91E0A1F1B1FE0920705F09208050093FA
:108C6000090510930A0571E0E7167AEFF70670E040
:108C7000070770E017070CF475C480E09AEFA0E0D6
:108C8000B0E08093070590930805A0930905B09381
:108C90000A05E12C4AEFF42E012D112D8090A90335
:108CA0009090AA039401442737FD4095542FC801A2
:108CB000B7010E94C1610091DE081091DF08020F28
:108CC000131FC10137FE02C00C94C25095958795C1
:108CD000860D971D5C01CC24B7FCC094DC2C9091D0
:108CE000BA0399A3292F30E040E050E0C601B50156
:108CF0000E944D6120E430E040E050E00E94C161FC
:108D0000C901021713070CF4980144245524481A8A
:108D1000590A421653060CF429018091A20490913D
:108D2000A30428A539A5281B390B3093BE0820932E
:108D3000BD08AFA1AA2309F4B9C2E981FA81E81BF1
:108D4000F90BCF01AA2797FDA095BA2FE090030554
:108D5000F09004050091050510910605E80EF91E36
:108D60000A1F1B1FE0920305F092040500930505FE
:108D700010930605F1E0EF16FAEFFF06F0E00F079B
:108D8000F0E01F070CF4D0C380E09AEFA0E0B0E061
:108D90008093030590930405A0930505B093060501
:108DA000E12C9AEFF92E012D112D9401442737FD66
:108DB0004095542FC801B7010E94C1610091BD08C0
:108DC0001091BE08020F131F69A1262F30E040E06A
:108DD00050E0C601B5010E944D6120E430E040E062
:108DE00050E00E94C161A901E22F232F041715074B
:108DF0001CF4C801E02F292F66277727641B750B09
:108E00008E2F922F861797070CF4CB01ADE5B5E0B6
:108E10002296BFAFAEAF22970DE0802E09E0902ED4
:108E20001EEEC12E18E0D12E9101442737FD40954A
:108E3000542F2CAB3DAB4EAB5FABA301662757FD68
:108E40006095762F48AF59AF6AAF7BAF9201442748
:108E500037FD4095542F2CAF3DAF4EAF5FAF2C0187
:108E6000662457FC6094762C3FA5232E33248BC0B8
:108E700013962C91332727FD3095432F532F6CA940
:108E80007DA98EA99FA90E944D6120E430E040E0B9
:108E900050E00E94C16179018A012A2D332727FD04
:108EA0003095432F532F68AD79AD8AAD9BAD0E94AD
:108EB0004D6120E430E040E050E00E94C161E20EEC
:108EC000F31E2296EEADFFAD22972181332727FDB9
:108ED0003095432F532F6CAD7DAD8EAD9FAD0E946D
:108EE0004D6120E430E040E050E00E94C161E20EBC
:108EF000F31E2296AEADBFAD229712962C9133276A
:108F000027FD3095432F532FC301B2010E944D61BD
:108F100020E430E040E050E00E94C161E20EF31E28
:108F2000F60160817181C7010E94CB2CD6018C9320
:108F300011969C9397FD9EC1AC015595479555950B
:108F400047958091D308282F30E0421753072CF023
:108F50009101421553050CF49A01F40120832296E5
:108F6000EEADFFAD229734962296FFAFEEAF22977B
:108F70000894811C911C22E030E0C20ED31EED58F3
:108F8000F54009F479C12296AEADBFAD2297AC9001
:108F90001A140CF46DCFD4011C92E1CF80919F0480
:108FA0008D3810F40C94043F1092920480917B0849
:108FB00022E3829FC00111249093EE048093ED047C
:108FC000ED81FE81B9979CF08091A804882379F007
:108FD0008091C9049091CA04FFEF8F3F9F0711F45D
:108FE0000C94995101969093CA048093C90480917E
:108FF000C9049091CA048F3F910519F010F00C94A8
:1090000099511092070510920805109209051092C7
:109010000A0510920305109204051092050510929E
:1090200006058A3F910511F40C947C5480916208E6
:10903000A82FB0E0AA0FBB1FFD01E25DF74F8081B2
:109040009181813591050CF4C6C08091A8048823D4
:1090500009F0C1C080916308E82FF0E0EE0FFF1F18
:10906000E25DF74F808191818C34910514F40C946A
:109070000F538091EC048F5F8093EC04893C08F4DB
:10908000AAC04C3010F00C94CE5629981092A80427
:109090001092EC041092CA041092C90480916008E6
:1090A000482F50E0440F551FFA01E25DF74F8081D1
:1090B00091818734910514F40C94B956809161081C
:1090C000A82FB0E0AA0FBB1FFD01E25DF74F808122
:1090D00091818734910534F0FA01E25DF74F0190F8
:1090E000F081E02DFD01E25DF74F808191818734B1
:1090F000910514F40C94B656FA01E25DF74F8081A5
:1091000091818734910514F40C94B65622E0FD0148
:10911000E25DF74F80819181863491054CF4FA012C
:10912000E25DF74F80819181873491050CF023E057
:10913000FD01E25DF74F808191818A5B9F4F4CF486
:10914000FA01E25DF74F80819181873491050CF03F
:1091500024E0A25DB74F8D919C918A5B9F4F4CF4A8
:10916000425D574FDA018D919C91863491050CF444
:1091700025E0822F0E94E603E0916108F0E0EE0F07
:10918000FF1FE25DF74F0190F081E02DF7FF02C075
:109190000C94FF567E9714F00C947656E09160087C
:1091A000F0E0EE0FFF1FE25DF74F808191818A5B57
:1091B0009F4F14F00C94765681E08093FB0688EE66
:1091C00093E09093EF038093EE0380916208A82FC1
:1091D000B0E0AA0FBB1FA25DB74F8D919C918B5A37
:1091E0009F4F14F00C94043FE0916308F0E0EE0F01
:1091F000FF1FE25DF74F80819181855B9F4F14F0E7
:109200000C9420528091EB048F5F8093EB04893C97
:1092100010F00C94DB53E0916308F0E0EE0FFF1FB9
:10922000E25DF74F808191818C34910514F40C94A8
:109230002B528091EA048F5F8093EA04893C10F4FA
:109240000C94043F1092A80488EC8093EA041092D6
:10925000CA041092C9040C94043F8091870890E0DE
:109260002D813E81821793070CF4B9C181E0809370
:1092700094040DC8039660CECF5BDF4F0FB6F89411
:10928000DEBF0FBECDBFCF91DF911F910F91FF9039
:10929000EF90DF90CF90BF90AF909F908F907F9096
:1092A0006F905F904F903F902F900895C901AA272B
:1092B00097FDA095BA2FE0900305F090040500916A
:1092C000050510910605E80EF91E0A1F1B1FE09206
:1092D0000305F092040500930505109306054ACD99
:1092E000C901AA2797FDA095BA2FE0900705F09035
:1092F00008050091090510910A05E80EF91E0A1FDC
:109300001B1FE0920705F0920805009309051093D2
:109310000A05A9CCB7013FEF603B73070CF473C19A
:10932000613571050CF45CCC60E570E059CC29988E
:109330000C948B3E5EA1552309F47BC11092AE04C0
:109340001092AD041092B0041092AF0410929404E5
:109350002091E0083091E1084091E2085091E30843
:109360002D8F3E8F4F8F58A32090E7083090E8084C
:109370004090E9085090EA081C8A3091ED083FA31C
:10938000332341F41092AE041092AD041092B00455
:109390001092AF044D8D5E8D6F8D78A14093D004F7
:1093A0005093D1046093D2047093D3042092CC04E0
:1093B0003092CD044092CE045092CF0410926004BB
:1093C000109261041092620410926304109264047B
:1093D000109265041092660410926704109268045B
:1093E0001092690410926A0410926B041092E008C3
:1093F0001092E1081092E2081092E3081092E70838
:109400001092E8081092E9081092EA081092D50824
:109410001092D6081092D7081092D8081092C70858
:109420001092C8081092C9081092CA081092180425
:1094300010921704E090A404F090A504C701F7FE71
:109440004DC8882799278E199F0948C82296AEAD26
:10945000BFAD2297A853BF4F0CF0C9C988E39FEF57
:109460009093CD088093CC0822969FAF8EAF229721
:10947000BEC96FEF283336070CF0A3C988E39FEF0E
:109480009093C2088093C10828E33FEF9AC95FA177
:10949000652F70E080E090E028A939A94AA95BA96E
:1094A0000E944D6128EF3AE240E050E00E94C16125
:1094B0003A832983190175C93FA1632F70E080E0C9
:1094C00090E02D893E894F89588D0E944D6128EF8B
:1094D0003AE240E050E00E94C1613C832B833901B5
:1094E00058C9E0E08E16E0EC9E060CF06CCA80E0F5
:1094F00090EC90931C0980931B09812C70EC972EA3
:1095000062CA205B3C434F4F5F4F0CF05DC880EB5D
:109510009CE3AFEFBFEF8093800490938104A0930E
:109520008204B093830450C820E0E21626E0F206DD
:109530002FEF02072FEF12070CF037CC80E096E0F8
:10954000AFEFBFEF8093030590930405A09305054B
:10955000B0930605E12C86E0F82E8FEF082F8FEFF1
:10956000182F23CC80E0E81686E0F8068FEF080776
:109570008FEF18070CF092CB80E096E0AFEFBFEFD3
:109580008093070590930805A0930905B0930A05F9
:10959000E12C36E0F32E3FEF032F3FEF132F7ECB6E
:1095A000A0E0CA16A0ECDA060CF0FEC980E090EC50
:1095B0009093C0088093BF0899A788A7F5C980E059
:1095C000481680EC58060CF0E1C980E090EC9093CE
:1095D000CF088093CE08412CF0EC5F2ED7C99E8334
:1095E0008D8381E0809394040C944741BFEF2E3F1C
:1095F0003B070CF02EC62E5F3F4F3093A5042093FF
:10960000A4040C94D33F60EB7FEF613571050CF43B
:10961000E7CA8ACE930177FCA8C6359527956627B9
:109620007727621B730B6E157F050CF0D9CAB70143
:10963000D7CA6B89662309F081CE709194047C8B24
:10964000772309F07BCE80919008882309F476CEA9
:109650008091E0089091E108A091E208B091E308C0
:10966000BC01CD0120E031E040E050E00E94C1614A
:109670002F83388749875A872D8F3E8F4F8F58A366
:109680002093E0083093E1084093E2085093E30808
:109690002090E7083090E8084090E9085090EA08E8
:1096A000C201B10120E031E040E050E00E94C16120
:1096B0002B873C874D875E8719012A012093E70895
:1096C0003093E8084093E9085093EA08E090740862
:1096D000FF2400E010E0209160043091610440918B
:1096E000620450916304C801B7010E944D6120E0FB
:1096F00031E040E050E00E94C16159016A012093CD
:109700006004309361044093620450936304209199
:109710006404309165044091660450916704C80167
:10972000B7010E944D6120E031E040E050E00E942E
:10973000C16139014A012093640430936504409368
:109740006604509367046091680470916904809185
:109750006A0490916B0420E031E040E050E00E9408
:10976000C161209368043093690440936A04509364
:109770006B046F81788589859A856A197B098C09C4
:109780009D096093F3047093F4048093F50490931F
:10979000F604E0908F08FF2400E010E0A801970194
:1097A0000E94C16159016A012093E2043093E304ED
:1097B0004093E4045093E504C201B10166197709AE
:1097C000880999096093EF047093F0048093F10481
:1097D0009093F204A80197010E94C16179018A0166
:1097E0002093DE043093DF044093E0045093E104BF
:1097F000C601B50120E031E040E050E00E94C161C7
:109800003093B0042093AF04C801B70120E031E0E9
:1098100040E050E00E94C1613093AE042093AD045B
:109820008091C5049091C60481349105BCF4809167
:10983000C7049091C8048134910584F4E0916308D1
:10984000F0E0EE0FFF1FE25DF74F0190F081E02D99
:10985000F7FF02C00C9408577A9734F080918B0977
:109860008F3F11F40C949456298D3A8D4B8D5C8D5D
:109870006D897E898F89988D261B370B480B590B74
:109880002093FB043093FC044093FD045093FE04AA
:10989000EAA0FBA00CA11DA188A999A9AAA9BBA90E
:1098A000E81AF90A0A0B1B0BE092F704F092F8048D
:1098B0000093F9041093FA042093F3043093F40412
:1098C0004093F5045093F604E092EF04F092F00414
:1098D0000093F1041093F204809174049091750444
:1098E000A0917604B0917704821B930BA40BB50B67
:1098F0008093740490937504A0937604B0937704D6
:1099000080917C0490917D04A0917E04B0917F04AD
:109910008E199F09A00BB10B80937C0490937D045A
:10992000A0937E04B0937F0480919008882371F106
:1099300020919504309196042138310594F080915E
:109940003E0490913F04019690933F0480933E041F
:109950008091EB089091EC0801969093EC0880932D
:10996000EB0820583F4F94F480913E0490913F04BF
:10997000019790933F0480933E048091EB0890916F
:10998000EC0801979093EC088093EB0810929604F2
:109990001092950481E090E09093D9048093D804CC
:1099A000E090F304F090F4040091F5041091F604B3
:1099B000D801C70117FF02C00C94D65681509240BF
:1099C000A040B04034F084E090E09093D9048093BC
:1099D000D8048091D0049091D104A091D204B09188
:1099E000D3042F81388549855A85821B930BA40B9C
:1099F000B50B815E914BAF4FBF4F8F539C49A04039
:109A0000B04010F40C94965580918C09893114F073
:109A10000C9496551092D9041092D80488EE93E0D5
:109A20009093A00380939F03CC24DD248091900821
:109A300090E08C159D0524F49093D9048093D8046C
:109A400080918C09882379F0282F332727FD3095C2
:109A50008091D8049091D9042817390724F43093C1
:109A6000D9042093D80481E8E816F1040105110512
:109A700074F080913A0490913B042091D804309185
:109A8000D904820F931F90933B0480933A0490E88B
:109A9000E9169FEFF9069FEF09079FEF190774F486
:109AA00080913A0490913B042091D8043091D904DC
:109AB000821B930B90933B0480933A0481E090E0E7
:109AC0009093D9048093D804E090EF04F090F004D0
:109AD0000091F1041091F204D801C70117FF02C0F0
:109AE0000C94F45681509240A040B04034F084E091
:109AF00090E09093D9048093D8041092DE041092E1
:109B0000DF041092E0041092E1048091CC04909163
:109B1000CD04A091CE04B091CF042B853C854D851A
:109B20005E85821B930BA40BB50B815E914BAF4FEF
:109B3000BF4F8F539C49A040B04008F43AC7809172
:109B40008C0989310CF035C71092D9041092D804D1
:109B500088EE93E09093A00380939F03CC24DD24B0
:109B60008091900890E08C159D0524F49093D90481
:109B70008093D80480918C09882379F0282F33278B
:109B800027FD30958091D8049091D9042817390782
:109B900024F43093D9042093D80481E8E816F10422
:109BA0000105110574F080913C0490913D042091D1
:109BB000D8043091D904820F931F90933D04809371
:109BC0003C0490E8E9169FEFF9069FEF09079FEF25
:109BD00019070CF0D2CB80913C0490913D04209168
:109BE000D8043091D904821B930B90933D04809349
:109BF0003C04C3CB6D897E898F89988D20E032E04B
:109C000040E050E00E94C161890137FDB1C368A9FD
:109C100079A98AA99BA920E032E040E050E00E94A7
:109C2000C161390137FDA8C3601671060CF44CC33D
:109C3000A0902209B0902309C0902409D090250952
:109C40008091BD039091BE03A091BF03B091C0036A
:109C50008AA79BA7ACA7BDA780901B0990901C0961
:109C6000C40197FC8EC3813891050CF036C3ACE17A
:109C7000B2E04A0E5B1E72010027F7FC0095102F20
:109C8000E4EEFDEF4E0E5F1EC601B5012AA53BA511
:109C90004CA55DA50E94C161E21AF30A040B150BE5
:109CA000C801B70128E631E040E050E00E94C16100
:109CB000645B70401B01220C331C220C331C220CF1
:109CC000331C20919F033091A00322963FAF2EAF0B
:109CD0002297232B99F439E1631671047CF4809167
:109CE000950490919604860F971F90939604809305
:109CF00095048091E604882309F06DC4B30175953D
:109D0000679575956795759567956F5F7F4FC101ED
:109D10000E948C619B01442737FD4095542F2A0DEA
:109D20003B1D4C1D5D1D2093220930932309409358
:109D30002409509325098091AF03C82EDD246C9C23
:109D4000C0016D9C900D7C9C900D112497FD3FC42B
:109D500095958795959587959595879595958795EB
:109D6000959587955601A81AB90AB7FC57C322964C
:109D70006EAD7FAD2297672B09F045C36090C70495
:109D80007090C8048091C5049091C604680E791E35
:109D900077FC89C7759467947594679475946794F4
:109DA000A0E4B0E06A0E7B1E80918E0490918F0437
:109DB000AA2797FDA095BA2F1CE1E12E12E0F12E03
:109DC000012D112DE81AF90A0A0B1B0BCA01B90162
:109DD0002AA53BA54CA55DA50E94C161E20EF31E1C
:109DE000041F151FC801B70128E631E040E050E02C
:109DF0000E94C161645B70406A9DC0016B9D900DC3
:109E00007A9D900D1124B3010E948C61C601880FC8
:109E1000991F8C0D9D1D861797070CF4DAC34427F4
:109E20005527481B590B641775070CF4BA019B01A1
:109E3000442737FD4095542F8091800490918104F0
:109E4000A0918204B0918304820F931FA41FB51FB9
:109E50008093800490938104A0938204B093830440
:109E60000C94F54281E08093E6040C947C4280914E
:109E7000AC03823308F036C28091C20381508093D4
:109E8000C2038F5F11F00C941945809122039091C9
:109E90002303895E934008F014C5809122039091BA
:109EA00023038436910508F03CC587B5823008F459
:109EB00038C587B58B3008F453C790911404965F6A
:109EC000909314048091F107891B87BD8CE291E087
:109ED0009093EF038093EE038AEF8093C203209167
:109EE000A9043091AA040C941D452D813E81232B99
:109EF00011F40C94F04481E090E09093CA048093B4
:109F0000C9048091D308482F50E05E834D830C94A0
:109F1000F0448B89882311F00C9458428091E60715
:109F20009091E707815092400CF4D0C180918B0949
:109F30008F3F09F494C2E0907408FF2400E010E021
:109F4000A82EBB24A7FCB094CB2CDB2C6D897E897A
:109F50008F89988DA80197010E94C16180910A099B
:109F600090910B09AA2797FDA095BA2F281B390BB2
:109F70004A0B5B0BCA01B901A60195010E944D6114
:109F800020E032E040E050E00E94C1612F87388B32
:109F9000498B5A8B922E832E742E652E68A979A92F
:109FA0008AA99BA9A80197010E94C16180912609F5
:109FB00090912709AA2797FDA095BA2F281B390B46
:109FC0004A0B5B0BCA01B901A60195010E944D61C4
:109FD00020E032E040E050E00E94C161122F032FE8
:109FE000F42EE52E180127018091C5049091C60436
:109FF000813491050CF0CAC18091C7049091C804C6
:10A00000813491050CF0C2C1E0916308F0E0EE0FDD
:10A01000FF1FE25DF74F0190F081E02DF7FDBAC41C
:10A020007A97E4F0692D782D872D962D23E030E086
:10A0300040E050E00E94C161922E832E742E652E66
:10A04000632D722D852D942D23E030E040E050E00B
:10A050000E94C161322E232E542E452E60918D090F
:10A06000A62EBB24A7FCB094CB2CDB2C292D382D9D
:10A07000472D562DC901DA019C01AD01A216B30688
:10A08000C406D50614F4A6019501862F992787FDED
:10A090009095909581959F4F7C010027F7FC009546
:10A0A000102F39014A012E153F054007510714F4BE
:10A0B00037014801232D322D452D542DC901DA01D8
:10A0C000A816B906CA06DB0614F4D601C5018E151A
:10A0D0009F05A007B10714F07C018D0180917004E9
:10A0E00090917104A0917204B0917304861997093C
:10A0F000A809B9098093700490937104A093720425
:10A10000B09373048091780490917904A0917A04BB
:10A11000B0917B048E199F09A00BB10B809378043A
:10A1200090937904A0937A04B0937B040C945842E2
:10A1300001979093EE048093ED044A3011F00C9453
:10A14000C33E289A0C94C83E415050405093C804D6
:10A150004093C7040C947140415050405093C60442
:10A160004093C5040C9443401092A8040C94043FFF
:10A170006D5F7F4F0C94A842EE27FF27EE19FF0971
:10A180000C948E4288279927821993090C9466466D
:10A1900020916F0830E080910007992787FD909506
:10A1A000289FA001299F500D389F500D11248091A8
:10A1B000A0049091A104840F951F9093A104809313
:10A1C000A00480910107992787FD9095F901E89FE8
:10A1D0009001E99F300DF89F300D11248091A20469
:10A1E0009091A304820F931F9093A3048093A204E1
:10A1F00020910207332727FD30958091A404909188
:10A20000A504820F931F9093A5048093A40420912A
:10A210006D0830E080910407992787FD9095AC0187
:10A22000249FC001259F900D349F900D1124909381
:10A23000BC038093BB038091030790E080179107D4
:10A2400014F00C9407409093A7048093A6040C94F8
:10A2500007401092A5041092A4040C94D33F1092CE
:10A26000B1040C943C411092B2040C942B4181E057
:10A270008093B5040C941E4181E08093B6048091D4
:10A280008808482F50E061E00C94FA4081E0809308
:10A29000B40480918808482F50E00C94D34081E0AA
:10A2A0008093B3040C94AF4084E690E09093C8048C
:10A2B0008093C7040C94714084E690E09093C604A8
:10A2C0008093C5040C9443403801B2CC8091A8041B
:10A2D000882311F40C94584229CE60E070E02224C7
:10A2E0003324EFCC81E08093930488EC8093C20305
:10A2F0002091A9043091AA040C941D451092B60433
:10A3000080916008A82FB0E080918808482F50E025
:10A31000AA0FBB1F60E00C94FA401092B404809125
:10A320008808482F50E00C94D3401092B5040C9448
:10A330001E418091CB0482608093CB040C9416481C
:10A3400003960C942C432D5F3F4F0C943D4388E9BA
:10A350009AE39093EF038093EE0380E09CE0909368
:10A360001203809311030C94B33E2F5F3F4F55C9E6
:10A37000109501951F4F4BCC7094619471087394A4
:10A3800053CC88279927881999096DCC6F857889CE
:10A3900089899A8922E030E040E050E00E94C16162
:10A3A000922E832E742E652E612F702F8F2D9E2D51
:10A3B00022E030E040E050E00E94C161322E232EC6
:10A3C000542E452E21CE1092A7041092A6040C9470
:10A3D0000F40309521953F4F0C9459402D5F3F4FD2
:10A3E0000C945140309521953F4F0C942B402D5F9C
:10A3F0003F4F0C9423404D5F5F4F0C94353F4D5FB2
:10A400005F4F0C94893F2296EEADFFAD22973197B6
:10A41000F093A003E0939F030C94F54284EF91E046
:10A420009093A00380939F030C94F542309521955F
:10A430003F4F0C946340309521953F4F0C9435402D
:10A440001092EB040C940B496416750614F40C94EA
:10A45000B9450C94BD451092EA040C94043FE09079
:10A460007408FF2400E010E06D897E898F89988D43
:10A47000A80197010E94C16159016A0180910A09EE
:10A4800090910B09AA2797FDA095BA2FA81AB90A8F
:10A49000CA0ADB0A68A979A98AA99BA9A801970118
:10A4A0000E94C16179018A01809126099091270952
:10A4B000AA2797FDA095BA2FE81AF90A0A0B1B0BD9
:10A4C000C601B50120E130E040E050E00E94C161EA
:10A4D000D22EC32EB42EA52E822F932FA42FB52FAC
:10A4E0003C014D01C801B70120E130E040E050E0FF
:10A4F0000E94C161522E432E342E252E822F932F7F
:10A50000A42FB52F7C018D018091C5049091C604C4
:10A51000813491050CF4E7C16D2D7C2D8B2D9A2D86
:10A5200023E030E040E050E00E94C161C901DA015F
:10A530003C014D01652D742D832D922D23E030E0DB
:10A5400040E050E00E94C161C901DA017C018D0147
:10A55000E0916308F0E0EE0FFF1FE25DF74F01901E
:10A56000F081E02DF7FDBAC37A97C4F0C401B301BE
:10A5700023E030E040E050E00E94C161C901DA010F
:10A580003C014D01C801B70123E030E040E050E05C
:10A590000E94C161C901DA017C018D01B1E26B1633
:10A5A0007104810491040CF4E2C190E2692E712CD3
:10A5B000812C912CF1E2EF16F104010511050CF448
:10A5C000C3C110E2E12EF12C012D112D87CD4F9644
:10A5D000BFCBBC012CCC88EC90E09093EF03809330
:10A5E000EE03B201882777FD8095982F2AA53BA519
:10A5F0004CA55DA50E944D61162F072FF82EE92E60
:10A600000E94C16130938F0420938E041092E6045F
:10A61000812F902FAF2DBE2D5C016D016FCB8081FE
:10A620009181855B9F4F0CF043C38091EC048F5F59
:10A630008093EC04893C10F40C94EB484C3008F007
:10A64000DCC32998F999FECF1FBA04E010E012BDCF
:10A6500001BD8FEF80BD0FB6F894FA9AF99A0FBE3C
:10A660001092A8041092EC041092CA041092C9042B
:10A670000E94BD3B4091440450914504F999FECF9E
:10A680001FBA12BD01BD9A0157FDC7C3832F992779
:10A6900087FD9A9580BD0FB6F894FA9AF99A0FBE85
:10A6A000F999FECF1FBA85E090E092BD81BDCA0145
:10A6B00060E071E00E948C6180BD0FB6F894FA9A58
:10A6C000F99A0FBE4091460450914704F999FECF84
:10A6D0001FBA86E090E092BD81BDCA0157FDA3C3B9
:10A6E000892F990F990B80BD0FB6F894FA9AF99AB1
:10A6F0000FBEF999FECF1FBA87E090E092BD81BDF1
:10A70000CA0160E071E00E948C6180BD0FB6F894D0
:10A71000FA9AF99A0FBE20914A0430914B04409165
:10A720004C0450914D04F999FECF1FBA88E090E097
:10A7300092BD81BDCA01B9010E946660CB0177FD5F
:10A740006FC3892F990F990B80BD0FB6F894FA9AB1
:10A75000F99A0FBE20914A0430914B0440914C0469
:10A7600050914D04F999FECF1FBA89E090E092BD57
:10A7700081BDCA01B9010E946660DC01CB0160E0C5
:10A7800071E00E948C6180BD0FB6F894FA9AF99A34
:10A790000FBE0E94CB030E94453E80916208A82F05
:10A7A000B0E0AA0FBB1F0C94EB483093E904209350
:10A7B000E8040C94BD4588EC8093EB0481E090E0C4
:10A7C0009093CA048093C90481E08093A8041092F6
:10A7D000FF041092000510920105109202051092DC
:10A7E00080041092810410928204109283041092CB
:10A7F000840410928504109286041092870460915C
:10A800000A0970910B09882777FD8095982FE090B1
:10A810007408FF2400E010E0A80197010E944D6138
:10A820006093700470937104809372049093730426
:10A830006091260970912709882777FD8095982FC8
:10A840000E944D61609378047093790480937A0438
:10A8500090937B048091500490915104A0915204F4
:10A86000B09153048093740490937504A09376047C
:10A87000B09377048091580490915904A0915A04A0
:10A88000B0915B0480937C0490937D04A0937E043C
:10A89000B0937F04109207051092080510920905E5
:10A8A00010920A05109203051092040510920505F6
:10A8B000109206058091CB0488608093CB040C94A1
:10A8C0000B4987B58E3F08F0E8CA87B5843F08F08A
:10A8D0004AC2909114049A50909314048091F10705
:10A8E000891B87BDF3CA8091C7049091C804813445
:10A8F00091050CF42DCE10CE81E08093E6041092E9
:10A90000FF041092000510920105109202051092AA
:10A9100080041092810410928204109283040C949B
:10A9200016482091A9043091AA0424513040309354
:10A93000AC042093AB042C5E3F4F1092930481E053
:10A940008093C2030C941D4520EEE2162FEFF20611
:10A950002FEF02072FEF12070CF0C0CBB0EEEB2E5B
:10A96000BFEFFB2EBFEF0B2FBFEF1B2FB7CBE0EEE0
:10A970006E16EFEF7E06EFEF8E06EFEF9E060CF001
:10A9800019CE80EE682E8FEF782E8FEF882E8FEF06
:10A99000982E10CEF095E195FF4F42CB2F5F3F4FA1
:10A9A0000C9483454D5F5F4F0C9441450F960C947A
:10A9B0009A4541E0E41640E1F40640E0040740E037
:10A9C00014070CF484C18091D504882309F4FFC1D5
:10A9D000D801C70139E0B595A795979587953A9520
:10A9E000D1F7C090D804D090D904C80ED91ED09207
:10A9F000D904C092D804C801B70128E030E040E093
:10AA000050E00E94C161C901DA018093DE04909395
:10AA1000DF04A093E004B093E10489589341A0407F
:10AA2000B04064F088E893E1A0E0B0E08093DE04F9
:10AA30009093DF04A093E004B093E1046091DE04FE
:10AA40007091DF048091E0049091E10420E031E016
:10AA500040E050E00E94C1618091AD049091AE044D
:10AA6000820F931F9093AE048093AD0460E0E616CE
:10AA700060EFF6066FEF06076FEF16070CF023C1C5
:10AA80008091D404882309F4AAC188279927DC017E
:10AA90008E199F09A00BB10B29E0B595A795979545
:10AAA00087952A95D1F7C80ED91ED092D904C092A5
:10AAB000D804C801B70128E030E040E050E00E942F
:10AAC000C161C901DA018093DE049093DF04A09391
:10AAD000E004B093E10488579C4EAF4FBF4F64F43D
:10AAE00088E79CEEAFEFBFEF8093DE049093DF0426
:10AAF000A093E004B093E1046091DE047091DF0460
:10AB00008091E0049091E10420E031E040E050E0E9
:10AB10000E94C1618091AD049091AE04820F931F99
:10AB20009093AE048093AD040C94B04D41E0E416D4
:10AB300040E1F40640E0040740E014070CF4BCC018
:10AB40008091D704882309F43AC1D801C70159E09C
:10AB5000B595A795979587955A95D1F7C090D80444
:10AB6000D090D904C80ED91ED092D904C092D8046E
:10AB7000C801B70128E030E040E050E00E94C16128
:10AB8000C901DA018093E2049093E304A093E40402
:10AB9000B093E50489589341A040B04064F088E840
:10ABA00093E1A0E0B0E08093E2049093E304A093EB
:10ABB000E404B093E5046091E2047091E3048091B1
:10ABC000E4049091E50420E031E040E050E00E9490
:10ABD000C1618091AF049091B004820F931F909354
:10ABE000B0048093AF0460E0E61660EFF6066FEF06
:10ABF00006076FEF16070CF075C08091D604882306
:10AC000009F4CFC088279927DC018E199F09A00B72
:10AC1000B10B49E0B595A795979587954A95D1F7DA
:10AC2000C80ED91ED092D904C092D804C801B70169
:10AC300028E030E040E050E00E94C161C901DA0143
:10AC40008093E2049093E304A093E404B093E504BA
:10AC500088579C4EAF4FBF4F64F488E79CEEAFEF30
:10AC6000BFEF8093E2049093E304A093E404B093D5
:10AC7000E5046091E2047091E3048091E404909112
:10AC8000E50420E031E040E050E00E94C1618091A5
:10AC9000AF049091B004820F931F9093B0048093FF
:10ACA000AF040C94164D87E090E0680E791E72C8D0
:10ACB0001092EC040C94EB481092D704C090D80486
:10ACC000D090D90490CF1092D4040C94B04D10922F
:10ACD000D504C090D804D090D904C8CEF095E195A1
:10ACE000FF4F42CC1092D6040C94164D0E94CB0319
:10ACF00060E678E04DE50E948B048091680880FF53
:10AD000010C08091220390912303875B934038F415
:10AD100080912203909123038E5E924010F40E9452
:10AD200075200E94BD3B35CD8091AF049091B00459
:10AD30009C0137FD7EC0359527953093B004209354
:10AD4000AF048091AD049091AE049C0137FD6EC0BC
:10AD5000359527953093AE042093AD040C94344C74
:10AD600081E087BDB3C88EEF87BDB0C821E00C94E9
:10AD7000874880916108A82FB0E0AA0FBB1FFD0192
:10AD8000E25DF74F0190F081E02DF7FD3DC0E73423
:10AD9000F10514F40C94BC480C946448299A0C9462
:10ADA000464881E08093D6040C94164D8827992755
:10ADB000DC018E199F09A00BB10B0C94DE4C81E0D5
:10ADC0008093D704C090D804D090D9040CCF81E0F0
:10ADD0008093D504C090D804D090D90447CE81E0A8
:10ADE0008093D4040C94B04D88279927DC018E19E8
:10ADF0009F09A00BB10B0C94724D299A23CCF095AE
:10AE0000E195FF4F0C94CA48F095E195FF4FBFCFF5
:10AE1000F095E195FF4F0C942C4C21503F4F36CCD0
:10AE200081509F4F8ECC81509F4F5ACC2F5F3F4F08
:10AE30008FCF2F5F3F4F7FCF88EE809368083EE132
:10AE4000309369088BEF80936B088AE080936C08DD
:10AE500030936A0830936E0893E090936D0858E041
:10AE600050936F0820E12093700866E060937108AA
:10AE70005093720886EE809373083093740880E8CC
:10AE80008093750844E64093760888E780937708B6
:10AE9000909378088EE58093790883E280937A080E
:10AEA00084E180937B0810927C0820937D081092A7
:10AEB0007E0810927F0810928008109281081092EC
:10AEC000920810929308109294081092950840935B
:10AED000820888E2809383081092AC0892E39093F2
:10AEE000840886E98093850885E08093860890939E
:10AEF00087082AE520938808909389081092AB0868
:10AF000020938A0883E480938B0886E480938C08DE
:10AF100085E580938D0880938E0880E280938F086A
:10AF200080939008909391088FE58093960883EF23
:10AF30008093980830939708309399088DEF809309
:10AF40009A0840939B0820939C0820939D08209387
:10AF50009E088BE480939F088093A0088093A108AB
:10AF60001092A2086093A3085093A4082093A50808
:10AF70003093A6084093A7084093A80884E08093E4
:10AF8000A908A1EBB8E0E4E8F3E08CE001900D92B1
:10AF90008150E1F7089588E6809368085EE1509358
:10AFA00069088BEF80936B088AE080936C0850935C
:10AFB0006A0850936E0893E090936D088CE080933C
:10AFC0006F0880E18093700876E07093710868E004
:10AFD0006093720886EE809373085093740880E83B
:10AFE0008093750880E58093760888E780937708DA
:10AFF000909378088EE58093790883E280937A08AD
:10B0000050937B0810927C0830E230937D081092B8
:10B010007E0810927F08109280081092810810928A
:10B02000920810929308109294081092950844E6A2
:10B030004093820888E2809383081092AC0892E3E0
:10B040009093840886E98093850885E0809386083C
:10B05000909387082AE52093880890938908109296
:10B06000AB0820938A0883E480938B088CE3809359
:10B070008C0885E580938D0880938E0830938F0827
:10B08000309390089BE4909391088FE58093960805
:10B0900083EF8093980884E18093970880939908C0
:10B0A0008DEF80939A0840939B0820939C082093EF
:10B0B0009D0820939E0890939F089093A0089093DA
:10B0C000A1081092A2087093A3086093A40820938B
:10B0D000A5085093A6084093A7084093A80884E0C9
:10B0E0008093A908A1EBB8E0EEE8F3E08CE00190D2
:10B0F0000D928150E1F7089588E6809368083EE15B
:10B10000309369088BEF80936B088AE080936C081A
:10B1100030936A0830936E08E4E0E0936D085FE0D6
:10B1200050936F08309370088CE08093710878E03A
:10B130007093720886EE809373083093740880E8E9
:10B140008093750880E58093760826E92093770838
:10B1500083E0809378088EE58093790883E280937A
:10B160007A0830937B0810927C0860E260937D0837
:10B1700010927E0810927F08109280081092810829
:10B1800010929208109293081092940810929508C9
:10B1900044E64093820888E2809383081092AC08CA
:10B1A00092E3909384082093850885E08093860835
:10B1B000909387082AE52093880890938908109235
:10B1C000AB0820938A0883E480938B0810928C0844
:10B1D00085E580938D0880938E0880E180938F08A9
:10B1E00060939008409391088FE58093960883EFD1
:10B1F0008093980850939708509399088DEF809307
:10B200009A0840939B0820939C0820939D082093C4
:10B210009E088BE480939F088093A0088093A108E8
:10B220001092A20886E08093A3087093A40820934C
:10B23000A5083093A6084093A7084093A808E09378
:10B24000A908A1EBB8E0E6E9F3E08CE001900D92EB
:10B250008150E1F7089580912B0590912C05A091E4
:10B260002D05B0912E058093330590933405A0935E
:10B270003505B093360580912F0590913005A0914A
:10B280003105B09132058093370590933805A0932E
:10B290003905B0933A0508951092240510922305BC
:10B2A0001092260510922505089584B1806A84B90C
:10B2B0003D9A82E58CBD1DBC459A81E080932C09A6
:10B2C0008AEA8093300983E8809331098AE0809389
:10B2D00032091092340910923309109236091092F3
:10B2E000350910928E0910925209109253098AE47E
:10B2F0008093540983E08093550986E08093560932
:10B300000895EF92FF920F931F93F894E0907408C2
:10B31000FF24EE0CFF1CEE0CFF1C0027F7FC009531
:10B32000102F6091500470915104809152049091BB
:10B330005304A80197010E94C161309334092093FE
:10B340003309609158047091590480915A04909186
:10B350005B04A80197010E94C161309336092093D4
:10B3600035096091220970912309809124099091F7
:10B3700025092AE030E040E050E00E944D61209134
:10B38000BD033091BE034091BF035091C0030E94A2
:10B39000C16130933C0920933B09E0914804F0914E
:10B3A00049048091E4089091E508BF010E948C61F6
:10B3B000CB01880F991F860F971F9C01220F331F07
:10B3C00096FD2DC1359527953595279530933809EC
:10B3D0002093370980911E0990911F09BF010E9497
:10B3E0008C61CB01880F991F860F971F9C01220F3C
:10B3F000331F96FD11C135952795359527953093C7
:10B400003A09209339091092490410924804109285
:10B41000E5081092E40810921F0910921E0980910D
:10B4200032098C3009F497C18D3008F46CC08D302E
:10B4300009F422C18E3009F40AC17894809152092E
:10B44000882309F4DCC02091580930915909C901B9
:10B4500081509E4F8F5F934058F440915A0950910C
:10B460005B09CA0181509E4F8F5F934008F4DFC093
:10B4700080915E0990915F0921E08936920724F45A
:10B4800090938D0480938C0480918C0490918D0412
:10B49000845E9D4F20918E0430918F04821B930B0C
:10B4A00068E671E00E948C61845B90409093910407
:10B4B0008093900420916209309163098091EE039A
:10B4C0009091EF038217930728F48091FB0688235D
:10B4D00009F4A8C080915709873681F480916409E6
:10B4E00080938B098091650980938D09809166090D
:10B4F00080938C098091670980938E091F910F9129
:10B50000FF90EF9008958A3009F4E7C08B3009F07E
:10B5100094CFE0916208F0E0EE0FFF1FE25DF74F7D
:10B520000190F081E02D2FEFE138F20714F4E1E80B
:10B53000FFEFE038F10514F0EFE7F0E0E0934309A6
:10B54000E0916308F0E0EE0FFF1FE25DF74F01901E
:10B55000F081E02D4FEFE138F40714F4E1E8FFEF5C
:10B56000E038F10514F0EFE7F0E0E0934409E091F2
:10B570006108F0E0EE0FFF1FE25DF74F0190F081F0
:10B58000E02D6FEFE138F60714F4E1E8FFEFE03863
:10B59000F10514F0EFE7F0E0E0934509E091600871
:10B5A000F0E0EE0FFF1FE25DF74F0190F081E02D1C
:10B5B0008FEFE138F80714F4E1E8FFEFE038F10528
:10B5C00014F0EFE7F0E0E093460980919704809350
:10B5D0004709809199048093480980919B04809346
:10B5E000490980919D0480934A0980919F0480932A
:10B5F0004B09789480915209882309F024CF109246
:10B6000024051092230510922605109225051F91FE
:10B610000F91FF90EF9008952D5F3F4FECCE2D5F7F
:10B620003F4FD0CE3093EF032093EE0353CF809162
:10B63000680885FF1DCF3093240520932305509380
:10B640002605409325058AEF80933B0511CF809115
:10B650005309809343098091540980934409809150
:10B660005509809345098091560980934609809138
:10B67000080180934709E1CE80919A08809343099D
:10B6800080919B088093440980919C088093450990
:10B6900080919D088093460980919E088093470978
:10B6A0008091A208809348098091A308809349095A
:10B6B0008091A40880934A098091A70880934B0940
:10B6C0008091A50880934C098091A60880934D092C
:10B6D0008091A80880934E09B0CE8091B7048093E2
:10B6E00043098091B804809344098091B904809300
:10B6F00045098091BA04809346098091BB048093E8
:10B7000047098091BC04809348098091BD048093CF
:10B7100049098091BE0480934A098091CB048093AB
:10B720004B098091CB04837F8093CB0480911803D5
:10B730009091190380934C098091790880934D0969
:10B74000F999FECF82E090E092BD81BDF89A80B574
:10B7500080934E0972CE8091FB068630F0F01092F5
:10B76000FB0685E0809343098091A9049091AA0487
:10B7700090934609809345098091A90880934409D4
:10B7800080919F08809347098091A0088093480981
:10B790008091A1088093490950CE80934309E4CF5A
:10B7A00080912C09882309F43BC0459880E399E0F7
:10B7B00090932E0980932D0990913C05E92FF0E09C
:10B7C000ED53FC4F8081809332099F5F90933C053D
:10B7D000963010F010923C0510922C090E9481596D
:10B7E00081E080932F0900000000000000000000AD
:10B7F0000000000000000000000000000000000049
:10B800000000000000000000000000000000000038
:10B810000000000000008091300980934F098EBD28
:10B82000089580912C09882311F40DB407FE089522
:10B8300084E08093F003459A9EB580913E05813067
:10B8400009F459C0813008F03AC010925109909320
:10B850003D05913809F44BC020912F09203208F0A2
:10B860002AC0459800000000000000000000000011
:10B8700000000000000000000000000000000000C8
:10B8800000000000000000000000000000000000B8
:10B8900000000000E0912D09F0912E09E20FF11D4A
:10B8A00080818EBD90914F09890F80934F092F5F42
:10B8B00020932F09089581E080932C09F8CF8230DE
:10B8C00009F0CACF80915109E82FF0E0EF58F64F08
:10B8D00090838F5F809351098A31C0F080913D053C
:10B8E0009817D1F01092520910923E05B5CF81E021
:10B8F00080933E05B1CF9535B9F780913D058B5AC0
:10B9000080933D0582E080933E05A6CF80913D0562
:10B91000890F80933D05A0CFA7E5B9E0E1E7F9E005
:10B920008AE101900D928150E1F781E08093520904
:10B93000DBCF87B18C6087B942984398109243055A
:10B9400080E88093C903109244058093CA03089548
:10B95000809145058150809345058F5F09F04DC06A
:10B9600084E080934505809197088B3F08F046C09E
:10B97000809143058150809343058F5FA1F48091AE
:10B98000E6088150809343058091C903813009F412
:10B9900052C086958093C9038091C90390919608FF
:10B9A0008923B9F1429A809199088B3F60F0809188
:10B9B0001909873E30F08091980887FD36C043987A
:10B9C00008958A3070F18091440581508093440538
:10B9D0008F5F99F48091190981508093440580917B
:10B9E000CA03813021F186958093CA038091CA03EE
:10B9F000909198088923C9F4439808958091E608A6
:10BA0000873E48F48A3008F0B3CF8091960887FFCC
:10BA1000C9CF4298C8CF8091960887FDC3CF42987E
:10BA2000C2CF8091980887FDCACF439A089580E8D5
:10BA30008093CA03DBCF80E88093C903ADCF8091A8
:10BA4000C9008F778093C9008091C9008F7B809354
:10BA5000C9008091C9008F7D8093C9005A9A52987D
:10BA60001092CD0084E18093CC008091C800826068
:10BA70008093C80080E18093C9008091CA008F77CD
:10BA80008093CA008091CA008F7B8093CA00809106
:10BA9000CA008F7D8093CA008091CA008F7E8093F8
:10BAA000CA008091CA00877F8093CA008091C90034
:10BAB0008B7F8093C9008091CA0084608093CA0004
:10BAC0008091CA0082608093CA008091C80087FF7D
:10BAD00006C08091CE008091C80087FDFACF80918A
:10BAE000C90080688093C90008951F920F920FB615
:10BAF0000F9211240F931F932F933F934F935F93B4
:10BB00006F937F938F939F93AF93BF93CF93DF9365
:10BB1000EF93FF931091CE008091CB039091CC03D3
:10BB2000019709F462C080914605909147050E94F3
:10BB3000FF1690E020914E0530914F0521153105FB
:10BB4000B9F12130310509F4FFC02230310509F483
:10BB50000EC12330310509F471C081E090E090936B
:10BB6000CC038093CB0310924D0510924C0510929C
:10BB700049051092480587E090E00E94F5169093E1
:10BB8000470580934605FF91EF91DF91CF91BF91DB
:10BB9000AF919F918F917F916F915F914F913F9165
:10BBA0002F911F910F910F900FBE0F901F9018951E
:10BBB000892BA1F5C0914C05D0914D056097D8F225
:10BBC0008091480590914905892B11F410928303C7
:10BBD00010924D0510924C0510924905109248059F
:10BBE00010924F0510924E05C6CF1092CC031092C2
:10BBF000CB0387E090E00E94F51690934705809371
:10BC0000460510924D0510924C0510924F0510926A
:10BC10004E0510924B0510924A05B5CF81E090E099
:10BC200090934F0580934E05C0914C05D0914D05E2
:10BC30002196D0934D05C0934C05C0CF892B09F0B8
:10BC40008CCF82E090E090934F0580934E05C09199
:10BC50004C05D0914D052196D0934D05C0934C05D0
:10BC600020914A0530914B05F901F695E795F69537
:10BC7000E795EF70F0703196EB30F10508F09ECF4C
:10BC8000812F90E0322F2227822B932B93708050AC
:10BC9000924063E070E00E948C61AB018F01000F65
:10BCA000111FF801E25DF74F808191819B01281BF4
:10BCB000390BC90137FD9AC0069754F480919F044F
:10BCC000883C08F08CC080919F04865F80939F041D
:10BCD000F801E25DF74F808191819C01220F331FB3
:10BCE000280F391F240F351F37FD7DC03595279547
:10BCF00035952795CA010196821793070CF066C007
:10BD00002150304080919F04843B08F459C0F801D1
:10BD1000E25DF74F80819181A901481B590BCA014F
:10BD200063E070E00E948C61CB01880F991F860F41
:10BD3000971FF801EC5BF74F91838083025D174FEB
:10BD4000F801318320833ACF009709F0FECE82E0DC
:10BD500090E090934F0580934E05C0914C05D09193
:10BD60004D052196D0934D05C0934C0527CF0097E4
:10BD700009F0EFCE10934A0510924B0520914C0527
:10BD800030914D052230310571F083E090E09093C1
:10BD90004F0580934E05C901019690934D05809300
:10BDA0004C05EC010BCF109249051092480517FF86
:10BDB000ECCF81E090E09093490580934805E5CF72
:10BDC000F801EC5BF74F11821082B8CF4150504020
:10BDD000241735070CF096CF2F5F3F4F93CF88EC99
:10BDE00080939F0475CF2D5F3F4F80CF90958195B5
:10BDF0009F4F62CFCF93DF9380E197E20E94F516C9
:10BE0000EC018091C9008F778093C9008091C900AF
:10BE10008F7E8093C9005A9800D00F92EDB7FEB77D
:10BE2000118287EF96E0938382830E94E2120F9043
:10BE30000F900F90CE010E94FF16882309F083C057
:10BE40004A9BF8CF8AE590E00E94F516EC0100D0FD
:10BE50000F92EDB7FEB7118281EF96E09383828354
:10BE60000E94E212529A0F900F900F90CE010E9402
:10BE7000FF168823D9F380E090E05A9A0196843621
:10BE80009105D9F780E090E05A980196F1E0803969
:10BE90009F07D1F780E090E05A9A01968A30910589
:10BEA000D9F780E090E05A9801968A309105D9F749
:10BEB00080E090E05A9A019621E080399207D1F70C
:10BEC00080E090E05A980196E1E080399E07D1F732
:10BED00080E090E05A9A01968A309105D9F780E087
:10BEE00090E05A9801968A309105D9F780E090E069
:10BEF0005A9A0196F1E080399F07D1F780E090E0EF
:10BF00005A98019621E080399207D1F780E090E0BD
:10BF10005A9A01968A309105D9F780E090E05A98B4
:10BF200001968A309105D9F780E090E05A9A0196FF
:10BF3000E1E080399E07D1F752985A980E941F5D20
:10BF4000DF91CF91089500D00F92EDB7FEB7118227
:10BF500086EE96E0938382830E94E2120F900F9008
:10BF60000F9052985A980E941F5DDF91CF910895CB
:10BF7000FC014150504030F001900616D1F7319746
:10BF8000CF010895882799270895A0E0B0E0EBEC51
:10BF9000FFE50C94E6617C01EB018A01690109C0AF
:10BFA000CE012196F6010995F70181937F01015099
:10BFB000104001151105A1F7CDB7DEB7E8E00C94EC
:10BFC0000262A0E0B0E0E7EEFFE50C94E661EC0170
:10BFD0007B018A01690109C0CE012196F7016191B7
:10BFE0007F01F60109950150104001151105A1F7D7
:10BFF000CDB7DEB7E8E00C9402625058BB27AA2701
:10C000000ED00DC1FED030F003D120F031F49F3FAF
:10C0100011F41EF4F3C00EF4E095E7FBE9C0E92F3C
:10C020000FD180F3BA17620773078407950718F0DA
:10C0300071F49EF527C10EF4E0950B2EBA2FA02DBA
:10C040000B01B90190010C01CA01A0011124FF27C5
:10C05000591B99F0593F50F4503E68F11A16F040C0
:10C06000A22F232F342F4427585FF3CF46953795BF
:10C070002795A795F0405395C9F77EF41F16BA0B84
:10C08000620B730B840BBAF09150A1F0FF0FBB1F32
:10C09000661F771F881FC2F70EC0BA0F621F731F7B
:10C0A000841F48F4879577956795B795F7959E3FD8
:10C0B00008F0B3CF9395880F08F09927EE0F979566
:10C0C0008795089571D008F481E0089504D06894AC
:10C0D000B111D9C00895BCD088F09F5790F0B92F06
:10C0E0009927B751A0F0D1F0660F771F881F991FCD
:10C0F0001AF0BA95C9F712C0B13081F0C3D0B1E0DF
:10C100000895C0C0672F782F8827B85F39F0B93FEE
:10C11000CCF3869577956795B395D9F73EF49095CE
:10C120008095709561957F4F8F4F9F4F0895E8944C
:10C1300009C097FB3EF490958095709561957F4F6F
:10C140008F4F9F4F9923A9F0F92F96E9BB2793951D
:10C15000F695879577956795B795F111F8CFFAF42D
:10C16000BB0F11F460FF1BC06F5F7F4F8F4F9F4F5E
:10C1700016C0882311F096E911C0772321F09EE8BC
:10C18000872F762F05C0662371F096E8862F70E022
:10C1900060E02AF09A95660F771F881FDAF7880FFC
:10C1A0009695879597F90895990F0008550FAA0B52
:10C1B000E0E8FEEF16161706E807F907C0F01216BA
:10C1C0001306E407F50798F0621B730B840B950BBD
:10C1D00039F40A2661F0232B242B252B21F4089512
:10C1E0000A2609F4A140A6958FEF811D811D0895AF
:10C1F00097F99F6780E870E060E008959FEF80EC1A
:10C20000089500240A9416161706180609060895BC
:10C2100000240A9412161306140605060895092E22
:10C220000394000C11F4882352F0BB0F40F4BF2B91
:10C2300011F460FF04C06F5F7F4F8F4F9F4F0895D1
:10C2400057FD9058440F551F59F05F3F71F04795C7
:10C25000880F97FB991F61F09F3F79F087950895AC
:10C26000121613061406551FF2CF4695F1DF08C0CB
:10C27000161617061806991FF1CF869571056105E8
:10C2800008940895E894BB2766277727CB0197F990
:10C2900008958ADF08F48FEF0895629FD001739F9D
:10C2A000F001829FE00DF11D649FE00DF11D929F52
:10C2B000F00D839FF00D749FF00D659FF00D992791
:10C2C000729FB00DE11DF91F639FB00DE11DF91FB5
:10C2D000BD01CF0111240895991B79E004C0991F75
:10C2E000961708F0961B881F7A95C9F780950895D0
:10C2F000AA1BBB1B51E107C0AA1FBB1FA617B7078C
:10C3000010F0A61BB70B881F991F5A95A9F78095A7
:10C310009095BC01CD01089597FB092E07260AD000
:10C3200077FD04D0E5DF06D000201AF47095619502
:10C330007F4F0895F6F7909581959F4F0895A1E25C
:10C340001A2EAA1BBB1BFD010DC0AA1FBB1FEE1F8F
:10C35000FF1FA217B307E407F50720F0A21BB30BDA
:10C36000E40BF50B661F771F881F991F1A9469F756
:10C3700060957095809590959B01AC01BD01CF01B2
:10C38000089597FB092E05260ED057FD04D0D7DF60
:10C390000AD0001C38F450954095309521953F4FB8
:10C3A0004F4F5F4F0895F6F7909580957095619582
:10C3B0007F4F8F4F9F4F08952F923F924F925F92E2
:10C3C0006F927F928F929F92AF92BF92CF92DF92A5
:10C3D000EF92FF920F931F93CF93DF93CDB7DEB70A
:10C3E000CA1BDB0B0FB6F894DEBF0FBECDBF09949E
:10C3F0002A88398848885F846E847D848C849B84F5
:10C40000AA84B984C884DF80EE80FD800C811B8102
:10C41000AA81B981CE0FD11D0FB6F894DEBF0FBE31
:0AC42000CDBFED010895F894FFCFA1
:10C42A0051756164726F00000A010101FF6401C85D
:10C43A0000416E676C654E69636B202020202020C6
:10C44A0020416E676C65526F6C6C20202020202082
:10C45A00204163634E69636B202020202020202026
:10C46A0020416363526F6C6C202020202020202002
:10C47A00204779726F47696572202020202020208A
:10C48A002048696768742056616C756520202020F1
:10C49A00204163635A2020202020202020202020B1
:10C4AA0020476173202020202020202020202020C7
:10C4BA0020436F6D706173732056616C756520201F
:10C4CA0020566F6C74616765202020202020202070
:10C4DA0020456D7066616E67202020202020202074
:10C4EA00204779726F204B6F6D7061737320202023
:10C4FA00204D6F746F722046726F6E742020202058
:10C50A00204D6F746F7220526561722020202020A6
:10C51A00204D6F746F72204C656674202020202095
:10C52A00204D6F746F722052696768742020202032
:10C53A0020202020202020202020202020202020F1
:10C54A0020202020202020202020202020202020E1
:10C55A0020202020202020202020202020202020D1
:10C56A00204D4B334D61672043616C537461746590
:10C57A0020536572766F2020202020202020202042
:10C58A0020202020202020202020202020202020A1
:10C59A002020202020202020202020202020202091
:10C5AA002020202020202020202020202020202081
:10C5BA002020202020202020202020202020202071
:10C5CA002020202020202020202020202020202061
:10C5DA002020202020202020202020202020202051
:10C5EA00204B616C6D616E5F4D617844726966744F
:10C5FA002020202020202020202020202020202031
:10C60A00204E6176692053657269616C20446174B9
:10C61A00614750535F4E69636B2020202020202001
:10C62A00204750535F526F6C6C202020202020201E
:10C63A0020FFFFFC01FC01016400C409C409007D5C
:10C64A000000FF0373737301010203040506070860
:10C65A00090A48616C6C6F2057656C740000000011
:10C66A0000000000000000000000000000000000C0
:10C67A0000000000000000000000000000000000B0
:10C68A0000000000000000000000000000000000A0
:10C69A000000000000000000000000000000000090
:10C6AA0000000D01426567696E6E657200004E6F8B
:10C6BA00726D616C000053706F727400006400F454
:10C6CA000190D0030090D00300380130FB103A40AB
:10C6DA00089696020A64465A414064ECFF0B05002C
:0EC6EA000004640A0B0D0B0C0E010101000090
:00000001FF
